:1000000075817F7401F58F538EF1438E10C2D4C277
:04001000D302003ED9
:0300230002A355E0
:03002B0002A3909D
:0300330002A326FF
:10003B0002A304D291C2B7C2B6C2B57550FF7551B7
:10004B00FFD2A1D2B2D2B3C2167541FF75427FC2A5
:10005B0017C218C219C21AC21BC21CC21DC21EC2B1
:10006B001FC220C221C222D223D224D225D226D211
:10007B0027D228D229D22AD22BD22CD22DD22EC2A1
:10008B0054C253D253C232C256C257D233D247C2D2
:10009B0036C237C258C259C25EC25DC238C239C2FB
:1000AB000CC24DD23AD23BC23C756C00756D0075DB
:1000BB006F00756E0075717F75707FC24AC24BD22F
:1000CB004CD24EC24F756700756800C209C20EC292
:1000DB000BD20DC20F75690075440075450075464E
:1000EB0000754700754800754900754A00754B004F
:1000FB00754C00754D00754E00754F00D212D21322
:10010B00755B00755C00755D00755E007561007553
:10011B0062007563007564007573067574007576FF
:10012B0006757700754318757901757A017400901F
:10013B00003FF0900040F0743E900041F07400904E
:10014B000072F0900073F0900074F0900075F090D6
:10015B000076F07401900161F0900162F090016300
:10016B00F07400900160F0900164F07401900168EC
:10017B00F0900166F0900167F090016EF0900169CC
:10018B00F090016AF090016BF090016CF090016DB2
:10019B00F0900170F090016FF0900172F090068A70
:1001AB00F012965D9001C27400F074F0900182F031
:1001BB00749F900183F074C3900199F074039001C4
:1001CB009AF09006DA7400F07417900077F07405CB
:1001DB00900078F0740F900079F07401900171F039
:1001EB007400900135F0900136F0900137F09001DA
:1001FB0038F0900139F090013AF012968E129697E2
:10020B001296A01296A91296C412963E74009002F2
:10021B0001F0740090029AF012964A74009004B6A2
:10022B00F0740090054FF0740C79FF90029BF0A3D3
:10023B00F0D9FC740C79FF90039BF0A3F0D9FC74FC
:10024B000090049BF0740090049CF0740C79FF9068
:10025B000550F0A3F0D9FC7400900650F074009098
:10026B000651F074009006BCF074009006C6F09036
:10027B0006C7F09006C8F09006C9F09006CAF09039
:10028B0006CBF09006CCF09006CF7400F0126617F8
:10029B0012664C7550FF7551FF127E21755200127C
:1002AB0090641289FD753D0012A2DD12A2FA12A212
:1002BB009B5350DF128BDB128CFF7550FF7551FF78
:1002CB00128B5C128E1B128E2B122D691237AD7492
:1002DB0002900167F01248197403900167F01248FD
:1002EB00197404900167F01248197405900167F0B6
:1002FB001248197406900167F0124819740790019F
:10030B0067F01248197408900167F01248197401CC
:10031B00900167F01248199001E8E0A2E19250A217
:10032B00E2925A128DDE9001E3E09006CDF090013F
:10033B00E4E09006CEF01228C1122B25122AD0121F
:10034B0087E59001E57400F012A28D12A25C1210E9
:10035B0093020359783279FF0000D9FCD8F8227840
:10036B004B79FF0000D9FCD8F82278327932D9FECC
:10037B00D8FA22F87902D9F6D8F222E627F52C081A
:10038B0009E637F52D782C22C3E697F52C0809E6FC
:10039B0097F52D782C22862C872E0809862D872FF2
:0E03AB00120426783122863108863208863305
:1003B900088634872E09872F1203C9782C793322AE
:1003C90075350075361012040B1203DC1203FFD5C4
:1003D90036F422C3E533952EE534952FE53594009F
:1003E900500122E533952EF533E534952FF534E5A3
:1003F900359400F53522B3E52C33F52CE52D33F58D
:100409002D22C3E53133F531E53233F532E53333A6
:10041900F533E53433F534E53533F53522E52C8507
:100429002EF0A4F53185F032E52D852FF0A4F533B2
:1004390085F034E52D852EF0A42532F532E53335E6
:10044900F0F533E5343400F534E52C852FF0A42597
:1004590032F532E53335F0F533E5343400F534223D
:10046900E582C4540FF9E583C46922E58203035484
:100479003FF9E583030354C069227A0CC297D2A3DA
:10048900A29633C933C9C2A3DAF2F8D29722C2A31A
:10049900C2973392A6D2A3DAF5C2A3120483E95410
:1004A90003F9227A0574E0120497F5838882227A87
:1004B9000574D8120497F5838882227A0574C012CC
:1004C9000497F5838882227A0574C8120497F58304
:1004D9008882227A0574D0120497F5838882227A59
:1004E9000574E8120497F5838882227A0574F0125C
:1004F9000497F5838882227A0574F8120497F583A4
:10050900888222C2B412051C1205691205B6D2B43A
:10051900C2B422A846A947E9540F44507A08C2A197
:10052900C2A33392A6D2A3DAF77A08E8C2A3339218
:10053900A6D2A3DAF7C2A3D2A1A844A945E9540FC8
:1005490044D07A08C2A1C2A33392A6D2A3DAF77A19
:1005590008E8C2A33392A6D2A3DAF7C2A3D2A12292
:10056900A84AA94BE9540F44507A08C2B2C2A3332E
:1005790092A6D2A3DAF77A08E8C2A33392A6D2A345
:10058900DAF7C2A3D2B2A84EA94FE9540F44D07AE0
:1005990008C2B2C2A33392A6D2A3DAF77A08E8C294
:1005A900A33392A6D2A3DAF7C2A3D2B222A848A94A
:1005B90049E9540F44507A08C2B3C2A33392A6D270
:1005C900A3DAF77A08E8C2A33392A6D2A3DAF7C26C
:1005D900A3D2B3A84CA94DE9540F44D07A08C2B3A9
:1005E900C2A33392A6D2A3DAF77A08E8C2A3339258
:1005F900A6D2A3DAF7C2A3D2B322F53775380078A9
:1006090037753B22753C00793B1203A18682088627
:100619008322F5377538007837753B44753C007986
:100629003B1203A1868208868322F5377538007844
:1006390037753B20753C00793B1203A186820886F9
:10064900832220A204753E002220A003D204227531
:100659003E0122E53EB53F04853E3F22B400152008
:10066900040A0540853E3FD206D20222C204853ED5
:100679003FD2062220040A1540853E3FD206D20306
:1006890022C204853E3FD20622E56B20E601229074
:1006990006CFE070030206B60206FFE56B20E6010D
:1006A900229006CFE070030207480207919006D016
:1006B900E01475F006A49006C3739001820207DA6C
:1006C9009001820207DA90018202080090018202F9
:1006D90008109001820207DA9001820207DA90017C
:1006E900820207DA9001820207DA9001820207DAB0
:1006F9009001820207DA9006D0E01475F006A49002
:10070900070C739001830207DA9001830207F390C3
:10071900018302086490018302086490018302083E
:0E0729002690018302082A9001830208319075
:10073700018302080090018302083B9001830208AD
:100747004E9006D1E01475F006A4900755739001FA
:10075700990207DA9001990207DA900199020800D5
:100767009001990208109001990207DA9001990205
:1007770007DA9001990207DA9001990207DA9001E6
:10078700990207DA9001990207DA9006D1E0147509
:10079700F006A490079E7390019A0207DA90019AD7
:1007A7000207F390019A02086490019A0208649084
:1007B700019A02082690019A02082A90019A0208D3
:1007C7003190019A02080090019A02083B90019A21
:1007D70002084E12086512087E1208971208B01216
:1007E70008C91208E21208FB12091422120865123E
:1007F700087E1208971208B02212086512087E12A6
:1008070008971208B01208C92212086512087E124A
:1008170008971208B01208C91208E21208FB221240
:1008270008652212086512087E2212086512087EE2
:100837001208972212086512087E1208971208B04C
:100847001208C91208E22212086512087E120897D8
:100857001208B01208C91208E21208FB2222E56B3F
:1008670030E108C21720230ED22322C22320170605
:10087700D217E0B2E7F022E56B30E208C218202475
:100887000ED22422C224201806D218E0B2E6F022A3
:10089700E56B30E308C21920250ED22522C2252098
:1008A7001906D219E0B2E5F022E56A30E108C21A6A
:1008B70020260ED22622C226201A06D21AE0B2E439
:1008C700F022E56A30E208C21B20270ED22722C297
:1008D70027201B06D21BE0B2E3F022E56A30E308CB
:1008E700C21C20280ED22822C228201C06D21CE0B7
:1008F700B2E2F022E56A30E508C21D20290ED229AE
:1009070022C229201D06D21DE0B2E1F022E56A309D
:10091700E708C21E202A0ED22A22C22A201E06D289
:100927001EE0B2E0F022E56A30E40630E611C23894
:100937002230380122D2389006CFE07400F02230FE
:10094700380122D2389006CFE07401F0229006CF0A
:10095700E07009E551C2E3D2E5F55122E551D2E352
:10096700C2E5F55122120A339006CFE070079001D5
:100977008212099A2290018312099A22120A33904D
:1009870006CFE0700790019912099A2290019A12F6
:10099700099A22E020E709E550D2E1F5500209ADB6
:1009A700E550C2E1F550E020E609E550D2E2F55006
:1009B7000209C0E550C2E2F550E020E509E550D252
:1009C700E3F5500209D3E550C2E3F550E020E4090E
:1009D700E550D2E6F5500209E6E550C2E6F550E0EB
:1009E70020E309E550D2E7F5500209F9E550C2E7DF
:1009F700F550E020E209E551D2E1F551020A0CE594
:100A070051C2E1F551E020E109E551D2E4F5510287
:100A17000A1FE551C2E4F551E020E009E551D2E7AC
:100A2700F551020A32E551C2E7F55122E550D2E409
:100A3700F550E551D2E0D2E2D2E6F55122B4FF03F8
:100A4700740022B4EB012250012274EB22B401019D
:100A5700225003740122B4EC012250012274EC22CB
:100A6700B4FF03740022B40C0122500122740C223B
:100A7700B40101225003740122B410012250012253
:100A8700741022B40101225003740122B40A012216
:100A9700500122740A22B40101225003740122B4C6
:0E0AA700200122500122742022B401012250AD
:100AB50003740122B41F0122500122741F22B401C4
:100AC50001225003740122B4080122500122740846
:100AD50022B40101225003740122B41101225001F4
:100AE50022741122B40101225003740122B47F0142
:100AF50022500122747F22B4FF03740022B4030143
:100B050022500122740322B4EB012250012274EB1E
:100B150022B40101225003740122B40A01225001BA
:100B250022740A22B40101225003740122B40C017B
:100B350022500122740C22B40101225003740122B7
:100B4500B4030122500122740322B401012250038F
:100B5500740122B4040122500122740422B401015B
:100B6500225003740122B40301225001227403228E
:100B7500B40101225003740122B40501225001225F
:100B8500740522B40101225003740122B403012229
:100B9500500122740322B40101225003740122B4CE
:100BA500030122500122740322B40101225003746F
:100BB5000122B4060122500122740622B401012249
:100BC5005003740122B4190122500122741922B470
:100BD5000101225003740122B42201225001227422
:100BE5002222B40101225003740122B40A012250C9
:100BF5000122740A22B40101225003740122B407B0
:100C05000122500122740722B4FF03740022B47E2E
:100C15000122500122747E22B40301225003740381
:100C250022B48F0122500122748F22B40101225077
:100C350003740122B4030122500122740322B4017A
:100C450001225003740122B40201225001227402D0
:100C550022B40101225003740122B4020122500181
:100C650022740222B40101225003740122B402014C
:100C750022500122740222B4010122500374012280
:100C8500B4030122500122740322B401012250034E
:100C9500740122B45F0122500122745F22B4FF085F
:100CA500B9000374FE22740022B4010122500374BA
:100CB5000122B4110122500122741122B401012232
:100CC5005003740122B4050122500122740522B497
:100CD5000101225003740122B40B01225001227438
:100CE5000B22B40101225003740122B57C0122506C
:100CF5000122E57C22B40101225003740122B43A99
:100D05000122500122743A22B401012250037401D8
:100D150022B4460122500122744622B40101225018
:100D250003740122B4800122500122748022B4018F
:100D350001225003740122B40701225001227407D5
:100D450022B40101225003740122B40C0122500186
:100D550022740C22B40101225003740122B40C0147
:100D650022500122740C22B4010122500374012285
:100D7500B40C0122500122740C22B401012250034B
:100D8500740122B417012250012274172230090977
:100D9500C209300A02C20AD20B22305F09C25F3093
:100DA5000A02C20AD20B22305015E56B30E610302C
:100DB500E003C20C22200C07D20CB20E120DC52284
:100DC500300E0AD20AD20ED20F5350DF22D20DC2F4
:100DD5000EC20B43502022900173E02414FA7400D4
:100DE5003400FB7537D0753812753913753A0078AC
:100DF500378A3B8B3C793B1203B1E6F54108E6F5B2
:100E05004222D211F5992011FD22B4F808300A02C8
:100E1500C20AD20B22B4FA0AD20AD20ED20F53500A
:0E0E2500DF22B4FC0AD20DC20EC20B435020D5
:100E330022B4FB09D20AD20ED20F5350DF22B4F0F0
:100E43000775670075680022B4F107756700756858
:100E53000022B4F20775670075680022B4F30F75BA
:100E630067007568002230500122120E0F2250F6DF
:100E7300E5692490F57EE9B57E08756701C251C224
:100E83005522E5692480F57EE9B57E08756801D2AF
:100E930051C25522E56924B0F57EE9B57E06756732
:100EA30001D2552230E70D75670075680022020EE6
:100EB300F6020F0C2055FA2051F4A967B90001225C
:100EC300A967B901050567F56522B90214056760CD
:100ED30008E565120F3AD24F22E565121038D24F5A
:100EE30022B903050567F56522B904067567010292
:100EF3000ED222A968B9000122A968B901070568C1
:100F0300F565020EDC75680122A967B9000122A903
:100F130067B901050567F57F22B902090567F9126B
:100F23000F3ED24F22B903050567F57F22B90406A8
:100F3300756701020F212212100522E57FB4140305
:100F4300020F50500122B41E0122400122C3941407
:100F530075F003A4900F5B73020F79020F82020FE7
:100F630090020FA0020FAF020FBF020FC8020FD6ED
:100F7300020FE6020FF5E9120C0D900177F022E95A
:100F830075F00C8404120CD490017AF022E975F008
:100F93000E8404120BE7900175F0D23222E975F04A
:100FA3000584120BC1900174F0D23222E975F00F5F
:100FB3008404120CC1900176F0D23222E9120C0D96
:100FC30090018EF022E975F00C8404120CD4900188
:100FD30091F022E975F00E8404120BE790018CF076
:100FE300D23222E975F00584120BC190018BF0D245
:100FF3003222E975F00F8404120CC190018DF0D2F6
:101003003222B42414C39424FF90020E12106FE012
:10101300D2E7F01287F0D2322250EAB40B01224019
:10102300FDC3940CFF9004C312108DE0D2E7F012BD
:1010330088A2D23222303A0122B42414C39424FF6A
:1010430090020E12106FE0C2E7F0128808D232222B
:1010530050EAB40B012240FDC3940CFF9004C31269
:10106300108DE0C2E7F01288BAD23222128654EF12
:10107300240C8582378583387837F53B753C0079B6
:101083003B120386868208868322128662021072CE
:1010930012999C1299CF129DE012A1D812A23F126D
:1010A300A25C1233E41286C2128746127E7D12902E
:1010B300801294A4124AAB1284F212661712270804
:1010C300120DAC3050139001E7E0B40306120D9FEC
:1010D3000210DC120DDC120D92126617200D0302B2
:1010E30010FEC20D9001E6E0B401030210F674FC99
:1010F300120E071211E8C2B7129363300F46C20FE4
:101103009001E6E0B4010302111274FA120E071201
:1011130011E8C24C12851B12571390049CE01490E3
:10112300049BF0125ED1900651E014900650F0E556
:1011330050C2E5F550D2B7121DAF12931B12119591
:10114300C24AC24B300A03021093200E03021194C9
:10115300200B03021194C20B9001E6E0B4010302D9
:10116300117AB4020874F8120E0702117AB25C30D5
:101173005C0574F8120E0720500B305A08B25B302E
:101183005B03021194121DC212209A12123912111A
:101193009522121DEE121EF81292D81220C61221A9
:0E11A300D01223727E011224071224B77E029E
:1011B1001224071224B77E031224071224B77E04D7
:1011C1001224071224B77E051224071224B77E06C3
:1011D1001224071224B77E071224071224B77E08AF
:1011E1001224071224B722435020121F161221EE97
:1011F1007400900077F0900135F0900137F0900184
:1012010038F090013AF075520012968E12969712AC
:1012110096A01296A912982B900188E014A3F012BF
:10122100987690019FE014A3F0C256C25790015FD7
:101231007400F0C25BC25C2212166212167712169B
:10124100911216BF1216D91216F312170D12172783
:1012510012174712176112177B1217951217AF1247
:1012610017C91217E31217FD12181722B4010490BF
:10127100007A22B4020490007C22B4030490007E20
:1012810022B4040490008022B4060490008222B4A7
:10129100080490008422B4090490008622B40C044E
:1012A10090008822B4100490008A22B412049000A5
:1012B1008C22B4180490008E22B420049000902255
:1012C100B4240490009222B4300490009422B440DB
:1012D1000490009622B448049000982290009A222B
:1012E100E01475F004A49012EB73EF021360EF02A7
:1012F100152EEF0213ADEF0213FAEF021447EF02BE
:101301001494EF0214E1EF02157BEF0215C8EF020E
:1013110016151475F004A490131C7390007A229092
:10132100007E22900082229000882290008E2290DE
:1013310000942290009A2290007C229000802290BA
:1013410000842290008A22900090229000962290A0
:1013510000862290008C2290009222900098221404
:1013610075F004A49013697390007B2290007F2292
:10137100900083229000892290008F229000952274
:1013810090009B2290007D22900081229000852276
:1013910090008B229000912290009722900087224A
:1013A10090008D2290009322900099221475F004F0
:1013B100A49013B67390009C2290009E229000A0EE
:1013C100229000A3229000A6229000A9229000ACB6
:1013D1002290009D2290009F229000A1229000A4C3
:1013E100229000A7229000AA229000A2229000A59C
:1013F100229000A8229000AB221475F004A490144E
:1014010003739000AD229000AF229000B1229000B2
:10141100B4229000B7229000BA229000BD22900021
:10142100AE229000B0229000B2229000B52290002E
:10143100B8229000BB229000B3229000B622900007
:10144100B9229000BC221475F004A490145073903A
:1014510000BE229000C0229000C2229000C52290BE
:1014610000C8229000CB229000CE229000BF229093
:1014710000C1229000C3229000C6229000C9229090
:1014810000CC229000C4229000C7229000CA229072
:1014910000CD221475F004A490149D739000CF2206
:1014A1009000D1229000D3229000D6229000D92220
:1014B1009000DC229000DF229000D0229000D22206
:1014C1009000D4229000D7229000DA229000DD22F1
:1014D1009000D5229000D8229000DB229000DE22DD
:1014E1001475F004A49014EA739000E0229000E2D5
:1014F100229000E4229000E7229000EA229000ED81
:10150100229000F0229000E1229000E3229000E579
:10151100229000E8229000EB229000EE229000E65B
:0E152100229000E9229000EC229000EF2214AC
:10152F0075F004A4901537739000F1229000F32208
:10153F009000F5229000F8229000FB229000FE22EE
:10154F00900101229000F2229000F4229000F622E6
:10155F009000F9229000FC229000FF229000F722C9
:10156F009000FA229000FD22900100221475F004E1
:10157F00A490158473900102229001042290010619
:10158F00229001092290010C2290010F229001124A
:10159F002290010322900105229001072290010A57
:1015AF002290010D22900110229001082290010B30
:1015BF002290010E22900111221475F004A49015AF
:1015CF00D1739001132290011522900117229001DF
:1015DF001A2290011D2290012022900123229001B6
:1015EF001422900116229001182290011B229001C3
:1015FF001E22900121229001192290011C2290019C
:10160F001F22900122221475F004A490161E7390CD
:10161F00012422900126229001282290012B229052
:10162F00012E229001312290013422900125229027
:10163F000127229001292290012C2290012F229024
:10164F0001322290012A2290012D22900130229006
:10165F0001332290007A7400F012183490007BE06E
:10166F0004B410027400F02290007CE004B4021065
:10167F007400F012188690007DE004B4100274001C
:10168F00F02290007EE004B403247400F0B2B7900F
:10169F00017EE0B40202C2B6900195E0B40202C22C
:1016AF00B51218D890007FE004B410027400F02235
:1016BF00900080E004B404107400F012192A900016
:1016CF0081E004B410027400F022900082E004B4B0
:1016DF0006107400F012197C900083E004B410021D
:1016EF007400F022900084E004B408107400F0122B
:1016FF0019CE900085E004B410027400F02290001F
:10170F0086E004B409107400F0121A20900087E0EC
:10171F0004B410027400F022900088E004B40C1698
:10172F007400F0E550B2E5F550121A72900089E09E
:10173F0004B410027400F02290008AE004B4101078
:10174F007400F0121AC490008BE004B410027400FD
:10175F00F02290008CE004B412107400F0121B16EB
:10176F0090008DE004B410027400F02290008EE01F
:10177F0004B418107400F0121B6890008FE004B4CA
:10178F0010027400F022900090E004B42010740056
:10179F00F0121BBA900091E004B410027400F02212
:1017AF00900092E004B424107400F0121C0C90000E
:1017BF0093E004B410027400F022900094E004B49B
:1017CF0030107400F0121C5E900095E004B410020B
:1017DF007400F022900096E004B440107400F012F0
:1017EF001CB0900097E004B410027400F022900037
:1017FF0098E004B448107400F0121D02900099E0B4
:10180F0004B410027400F02290009AE004B4601344
:10181F007400F0121DAF121D5490009BE004B41021
:10182F00027400F02290009C757C05121DA690009A
:10183F00AD757C07121DA69000BE757C09121DA602
:10184F009000CF757C0A121DA69000E0757C0B12DC
:10185F001DA69000F1757C0C121DA6900102757CDF
:10186F000D121DA6900113757C0E121DA69001245A
:10187F00757C0F121DA62290009D757C05121DA66A
:10188F009000AE757C07121DA69000BF757C0912E3
:0E189F001DA69000D0757C0A121DA69000E1D7
:1018AD00757C0B121DA69000F2757C0C121DA69076
:1018BD000103757C0D121DA6900114757C0E121D71
:1018CD00A6900125757C0F121DA62290009E757C99
:1018DD0005121DA69000AF757C07121DA69000C0C5
:1018ED00757C09121DA69000D1757C0A121DA6905B
:1018FD0000E2757C0B121DA69000F3757C0C121D79
:10190D00A6900104757C0D121DA6900115757C0E17
:10191D00121DA6900126757C0F121DA62290009F08
:10192D00757C05121DA69000B0757C07121DA69042
:10193D0000C1757C09121DA69000D2757C0A121D7E
:10194D00A69000E3757C0B121DA69000F4757C0C1F
:10195D00121DA6900105757C0D121DA69001167520
:10196D007C0E121DA6900127757C0F121DA62290CC
:10197D0000A0757C05121DA69000B1757C07121D87
:10198D00A69000C2757C09121DA69000D3757C0A25
:10199D00121DA69000E4757C0B121DA69000F57526
:1019AD007C0C121DA6900106757C0D121DA69001D2
:1019BD0017757C0E121DA6900128757C0F121DA6A1
:1019CD00229000A1757C05121DA69000B2757C07B2
:1019DD00121DA69000C3757C09121DA69000D4752A
:1019ED007C0A121DA69000E5757C0B121DA69000B9
:1019FD00F6757C0C121DA6900107757C0D121DA6A7
:101A0D00900118757C0E121DA6900129757C0F1280
:101A1D001DA6229000A2757C05121DA69000B3751F
:101A2D007C07121DA69000C4757C09121DA690009E
:101A3D00D5757C0A121DA69000E6757C0B121DA6AD
:101A4D009000F7757C0C121DA6900108757C0D1287
:101A5D001DA6900119757C0E121DA690012A757C8C
:101A6D000F121DA6229000A3757C05121DA69000D5
:101A7D00B4757C07121DA69000C5757C09121DA6B4
:101A8D009000D6757C0A121DA69000E7757C0B128E
:101A9D001DA69000F8757C0C121DA6900109757C91
:101AAD000D121DA690011A757C0E121DA690012B0C
:101ABD00757C0F121DA6229000A4757C05121DA623
:101ACD009000B5757C07121DA69000C6757C091295
:101ADD001DA69000D7757C0A121DA69000E8757C96
:101AED000B121DA69000F9757C0C121DA690010A13
:101AFD00757C0D121DA690011B757C0E121DA690F6
:101B0D00012C757C0F121DA6229000A5757C051267
:101B1D001DA69000B6757C07121DA69000C7757C9A
:101B2D0009121DA69000D8757C0A121DA69000E919
:101B3D00757C0B121DA69000FA757C0C121DA690DB
:101B4D00010B757C0D121DA690011C757C0E121DCE
:101B5D00A690012D757C0F121DA6229000A6757CF6
:101B6D0005121DA69000B7757C07121DA69000C822
:101B7D00757C09121DA69000D9757C0A121DA690C0
:101B8D0000EA757C0B121DA69000FB757C0C121DD6
:101B9D00A690010C757C0D121DA690011D757C0E75
:101BAD00121DA690012E757C0F121DA6229000A766
:101BBD00757C05121DA69000B8757C07121DA690A8
:101BCD0000C9757C09121DA69000DA757C0A121DDC
:101BDD00A69000EB757C0B121DA69000FC757C0C7D
:101BED00121DA690010D757C0D121DA690011E757E
:101BFD007C0E121DA690012F757C0F121DA6229032
:101C0D0000A8757C05121DA69000B9757C07121DE4
:0E1C1D00A69000CA757C09121DA69000DB750A
:101C2B007C0A121DA69000EC757C0B121DA6900071
:101C3B00FD757C0C121DA690010E757C0D121DA658
:101C4B0090011F757C0E121DA6900130757C0F1232
:101C5B001DA6229000A9757C05121DA69000BA75D1
:101C6B007C07121DA69000CB757C09121DA6900057
:101C7B00DC757C0A121DA69000ED757C0B121DA65F
:101C8B009000FE757C0C121DA690010F757C0D1239
:101C9B001DA6900120757C0E121DA6900131757C3E
:101CAB000F121DA6229000AA757C05121DA690008E
:101CBB00BB757C07121DA69000CC757C09121DA666
:101CCB009000DD757C0A121DA69000EE757C0B1240
:101CDB001DA69000FF757C0C121DA6900110757C43
:101CEB000D121DA6900121757C0E121DA6900132BE
:101CFB00757C0F121DA6229000AB757C05121DA6DC
:101D0B009000BC757C07121DA69000CD757C091246
:101D1B001DA69000DE757C0A121DA69000EF757C47
:101D2B000B121DA6900100757C0C121DA6900111C3
:101D3B00757C0D121DA6900122757C0E121DA690AE
:101D4B000133757C0F121DA6229000AC757C051219
:101D5B001DA69000BD757C07121DA69000CE757C4C
:101D6B0009121DA69000DF757C0A121DA69000F0CB
:101D7B00757C0B121DA6900101757C0C121DA69093
:101D8B000112757C0D121DA6900123757C0E121D80
:101D9B00A6900134757C0F121DA622E004B57C02BF
:101DAB007400F02290017EE0B40202D2B69001954D
:101DBB00E0B40202D2B522304A0BC24A90049CE036
:101DCB001490049BF022900179E0121313E0900120
:101DDB0035F0900179E0FF9006D01212E1E090010E
:101DEB0037F022121DD1900135E0B40003121DFC17
:101DFB0022900137E07012F990017DE0B403099055
:101E0B00049CE01490049BF0E904121E65227400FC
:101E1B00900137F0C248227400900135F022740013
:101E2B0090049BF022B40803021E385012F9900163
:101E3B0078E075F002A4141490729B93021E5CC39D
:101E4B009408F9900178E075F002A4141490729C38
:101E5B009323D9FDA2E0121E8622B40803021E6D45
:101E6B005008F9900182E0021E7DC39408F990019D
:101E7B0083E023D9FDA2E0121E8622400E90017C46
:101E8B00E014700122D24812569422D2481231B774
:101E9B007400900136F01256949006BCE02BF5734B
:101EAB00900177E06006121EC7021EBD122042127F
:101EBB001EE490017EE0B40102D2B622122042E56C
:101ECB0073B57403021EE45005C214021EDBD21458
:101EDB00121F23C21285737422D212E573F574128A
:101EEB000603C2AD858244858345D2AD229001366F
:101EFB00E0F57C900187E0B57C04121F162240FAB6
:101F0B00121F0F22900136E004F022122080900164
:101F1B007EE0B40102C2B62220142CE57412060333
:101F2B00C2AD858244858345D2ADE574C39573F507
:101F3B0079120603858259E58270037559018583F1
:101F4B005A055A121F7E22E574120603C2AD858212
:101F5B0044858345D2ADE573C39574F579120603B9
:101F6B00858259E582700375590185835A055A128A
:101F7B001F7E22900177E0FA7480C39AF543753780
:101F8B00F175384E753904753A00783785793B759C
:0E1F9B003C00793B1203B18637088638753951
:101FA90000753A00783785433B753C00793B12034D
:101FB900B18637088638753900753A007837900147
:101FC90073E02414F53B753C00793B1203B186821A
:101FD900088683C2AD85825BE5827003755B0185E6
:101FE900835C055C855B5D855C5ED2AD22D5590558
:101FF900D55A03D212227559FF2230120122201418
:1020090003022027121FF630120122E5442401F5AC
:1020190082E5453400F58385824485834522121F74
:10202900F630120122C3E5449401F582E545940096
:10203900F5838582448583452290029AE0700412D3
:1020490020802212982BF57090017FE0B4010FE5F2
:1020590070120633C2AD85824C85834DD2AD1220F4
:10206900807490120E07E5732424C2E7120E07E567
:1020790070120E07D23422203401227490120E07F6
:10208900E5742424C2E7120E077400120E07C23445
:1020990022304B0BC24B900651E014900650F022AF
:1020A900900190E0121313E0900138F0900190E054
:1020B900FF9006D11212E1E090013AF0221220A914
:1020C900900138E0B400031220D42290013AE07064
:1020D90012F9900194E0B40309900651E0149006B6
:1020E90050F0E90412213D22740090013AF0C249EE
:1020F900227400900138F0227400900650F022B446
:1021090008030221105012F990018FE075F002A422
:10211900141490729B93022134C39408F990018F8F
:10212900E075F002A4141490729C9323D9FDA2E0E7
:1021390012215E22B408030221455008F990019941
:10214900E0022155C39408F990019AE023D9FDA230
:10215900E012215E22400E900193E014700122D218
:1021690049125E5222D249123A047400900139F0A0
:10217900125E529006BCE02BF57690018EE0600667
:1021890012219F02219512231A1221BC900195E078
:10219900B40102D2B52212231AE576B57703021EDD
:1021A900E45005C2150221B3D2151221FBC21385D1
:1021B900767722D213E576F577120603C2AD8582CA
:1021C90046858347D2AD22900139E0F57C90019E86
:1021D900E0B57C041221EE2240FA1221E722900197
:1021E90039E004F022122358900195E0B40102C2AB
:1021F900B52220152CE577120603C2AD85824685E6
:102209008347D2ADE577C39576F57A1206038582C1
:102219005FE5827003755F01858360056012225650
:1022290022E577120603C2AD858246858347D2AD82
:10223900E576C39577F57A12060385825FE58270A4
:1022490003755F0185836005601222562290018E15
:10225900E0FA7480C39AF5437537F175384E7539CC
:1022690004753A007837857A3B753C00793B12034F
:10227900B18637088638753900753A00783785434D
:102289003B753C00793B1203B186370886387539AE
:1022990000753A007837900173E02414F53B753CDA
:1022A90000793B1203B18682088683C2AD858261BB
:1022B900E5827003756101858362056285616385C5
:1022C9006264D2AD22D55F05D56003D21322755F52
:0422D900FF2230139D
:1022DD0001222015030222FF1222CE30130122E526
:1022ED00462401F582E5473400F5838582468583D2
:1022FD0047221222CE30130122C3E5469401F58206
:10230D00E5479400F5838582468583472290054FE6
:10231D00E0700412235822129876F571900196E020
:10232D00B4010FE571120633C2AD85824E85834F20
:10233D00D2AD1223587491120E07E5762424C2E70C
:10234D00120E07E571120E07D235222035012274C7
:10235D0091120E07E5772424C2E7120E07740012BE
:10236D000E07C235227E0112239B7E0212239B7E15
:10237D000312239B7E0412239B7E0512239B7E0654
:10238D0012239B7E0712239B7E0812239B22900112
:10239D00AA1223C7E0121313E090013B1223C7F0DA
:1023AD009001AA1223C7E0FF9006D21223C7121282
:1023BD00E1E090014B1223C7F022C0E08582378502
:1023CD0083387837EE14F53B753C00793B12038664
:1023DD008682088683D0E022C0E0858237858338E7
:1023ED007837EE1475F002A4F53B753C00793B127D
:1023FD0003868682088683D0E02290013B1223C794
:10240D00E0B400031224152290014B1223C7E004FF
:10241D0012247022740090014B1223C7F022740015
:10242D0090013B1223C7F022B4080302243D50153E
:10243D00FF9001A21223C7E075F002A4141490724C
:10244D009B93022467C39408FF9001A21223C7E057
:10245D0075F002A4141490729C9323DFFDA2E01278
:10246D00249722B40803022478500BFF9001D31255
:10247D0023E5E002248EC39408FF9001D41223E5D6
:10248D00E023DFFDA2E0122497224001221224B0A6
:10249D00124A611224B074009001431223C7F01246
:1024AD0024DE22900167E0CEF0229001431223C773
:1024BD00E0F57C9001CB1223C7E0B57C0412252BEF
:1024CD002240FA1224D4229001431223C7E004F0D3
:1024DD0022BE010743520112257822BE0207435244
:1024ED000212258F22BE03074352201225A622BEBB
:1024FD0004074352041225BD22BE05074352401264
:10250D0025D422BE06074352081225EB22BE07072B
:10251D004352801226022243521012261922BE0166
:10252D00075352FE12263022BE02075352FD1226C9
:10253D004B22BE03075352DF12266622BE040753F9
:10254D0052FB12268122BE05075352BF12269C2232
:10255D00BE06075352F71226B722BE070753527F06
:10256D001226D2225352EF1226ED227499120E0723
:10257D007424120E077464120E079006DAE0D2E08E
:10258D00F0227499120E077425120E07746E120E36
:10259D00079006DAE0D2E1F0227499120E07743C2E
:1025AD00120E077478120E079006DAE0D2E2F022CE
:1025BD007499120E07743F120E07747F120E079056
:1025CD0006DAE0D2E3F0227499120E077430120E7F
:1025DD0007746E120E079006DAE0D2E4F0227499B9
:1025ED00120E07743B120E07747F120E079006DA57
:1025FD00E0D2E5F0227499120E07743D120E0774A5
:10260D007F120E079006DAE0D2E6F0227499120ED0
:10261D0007743E120E07747F120E079006DAE0D291
:10262D00E7F0229006DAE020E00122C2E0F0749992
:10263D00120E077424120E077400120E0722900654
:0E264D00DAE020E10122C2E1F07499120E07DA
:10265B007425120E077400120E07229006DAE02082
:10266B00E20122C2E2F07499120E07743C120E07BB
:10267B007400120E07229006DAE020E30122C2E377
:10268B00F07499120E07743F120E077400120E07A6
:10269B00229006DAE020E40122C2E4F07499120ED3
:1026AB00077430120E077400120E07229006DAE040
:1026BB0020E50122C2E5F07499120E07743B120E4D
:1026CB00077400120E07229006DAE020E60122C200
:1026DB00E6F07499120E07743D120E077400120E79
:1026EB0007229006DAE020E70122C2E7F074991284
:1026FB000E07743E120E077400120E07221229C722
:10270B00E56B30E7071227F012299C221227CC1217
:10271B0027DE12272122900166E01475F006A490A3
:10272B00272E739067FD02276A90680302276A9031
:10273B00680902276A90680F02276A9068150227BA
:10274B006A90681B02276A90682102278F9068277E
:10275B0002276A90682D02276A9068330227B40516
:10276B00A29000427B06128B349067CA05A29000A0
:10277B00487B0A128B349067CA05A29000527B10DB
:10278B00128B342205A29000427B05128B3490678A
:10279B00CA05A29000477B0B128B349067CA05A227
:1027AB009000527B10128B342205A29000427B10BA
:1027BB00128B349067CA05A29000527B10128B3497
:1027CB002220020122C205900166E004120B16F0D2
:1027DB00C2022220030122C205900166E014120BF3
:1027EB0016F0C20322E56B20E50122E56B30E60112
:1027FB0022E56A30E02130E12730E22730E3273051
:10280B00E52730E727E56B30E02530E10D30E204BA
:10281B0030E30A2202283D02284C02285B02286A78
:10282B000228790228880228970228A00228AF02E2
:10283B0028B89001727401F07401900166F00228BF
:10284B00C59001727401F07402900166F00228C504
:10285B009001727402F07403900166F00228C59027
:10286B0001727403F07404900166F00228C59001A4
:10287B00727401F07405900166F00228C590017224
:10288B007401F07406900166F00228C5740790017C
:10289B0066F00228C59001727401F074089001660D
:1028AB00F00228C57409900166F00228C5740A90DD
:1028BB000166F00228C5900166E0B401069067FD41
:1028CB0002290EB4020690680302290EB403030218
:1028DB00291CB40403022930B4050690681502299B
:1028EB000EB4060690681B02290EB4070302294496
:1028FB00B40806906827022958B4090690682D027F
:10290B00290E2212296C05A29000427B06128B34F1
:10291B002290680912296C05A29000427B06128B4B
:10292B00341229792290680F12296C05A29000426B
:10293B007B06128B341229792290682112296C059F
:10294B00A29000427B05128B341246B82290682766
:10295B0012296C05A29000427B05128B34124C108D
:10296B00222220080122200501229067EA223053FF
:10297B00069069CB0229912054069069C3022991D4
:10298B009069C702299105A29000477B04128B34F2
:10299B0022900166E01475F003A49029A973022A12
:1029AB00030235FD023B3D023D37023FB70241D4E6
:1029BB000246ED024C45024EA70252A6E56B30E7EC
:0E29CB0003C20722200704B208D2072220020E
:1029D9000122C205900168E004120B29F0900169F7
:1029E900F0C2022220030122C205900168E01412FC
:1029F9000B29F0900169F0C20322E56B20E5012261
:102A0900C2541287E5122B25122AD0300807122941
:102A1900D71229ED22900168E0B4010A122BA21203
:102A29002BB612855222B4020A1230031230171241
:102A3900855222B4030A1230A51230B912855222E6
:102A4900B4040A1230F212310412855222B4051F5D
:102A5900122C8A122CA312069212096C12092D1239
:102A690009549001727404F09001637401F022B466
:102A7900060A122EE8122EFC12855222B4070A12F7
:102A8900314812315A12855222B4080A1231F5120C
:102A9900320712855222B4090A1232B71232C91208
:102AA900855222B40A0A1232FF12331112855222B8
:102AB900B40B0A12334D1233611285522212339F1D
:102AC9001233B112855222900168E0B40104122B2D
:102AD900CA22B4020412302B22B403041230CD22CC
:102AE900B4040412311622B40504122D4522B40689
:102AF90004122F2822B4070412316C22B4080412DC
:102B0900321922B409041232DB22B40A0412332323
:102B190022B40B04123375221233C322900168E0E8
:102B29001475F006A4902B3273906A41022B7A90A7
:102B39006A4B022B7A906A55022B7A906A5F022BB4
:102B49007A906A69022B88906A73022B7A906A7D5F
:102B5900022B7A906A87022B7A906A91022B7A90DB
:102B69006A9B022B7A906AA5022B7A906AAF022B94
:102B79007A122B9605A29000487B0A128B342212F6
:102B89002B9605A29000487B05128B342220080160
:102B990022200501229067EA2220020122C2059023
:102BA9000174E004120BC1F0C202D23222200301E7
:102BB90022C205900174E014120BC1F0C203D23293
:102BC90022900174E01475F006A4902BD773906CD1
:102BD90039022C7F906C49022C7F906C59022C7F12
:102BE900906C69022C7F906C79022C7F906C890221
:102BF9002C7F906C99022C7F906CA9022C7F906C91
:102C0900B9022C7F906CC9022C7F906CD9022C7F61
:102C1900906CE9022C7F906CF9022C7F906D09026F
:102C29002C7F906D19022C7F906D29022C7F906D5D
:102C390039022C7F906D49022C7F906D59022C7FAF
:102C4900906D69022C7F906D79022C7F906D8902BD
:102C59002C7F906D99022C7F906DA9022C7F906D2D
:102C6900B9022C7F906DC9022C7F906DD9022C7FFF
:102C7900906DE9022C7F05A29000527B10128B34D3
:102C89002220020122C205900178E0F904120CA267
:102C9900F0C202122E4B122D692220030122C20515
:102CA900900178E0F914120CA2F0C203122E4B1213
:102CB9002D6922E0B48003022CD550FB122CE89038
:102CC9000050128B6D90004F7450F022C3947F1204
:102CD9002CE8900050128B6D90004F7455F022B47F
:102CE90020012240FDB43F04C394202240FAC3943A
:102CF9004075F00884E5F00422E01475F005A4900D
:102D09002D0C737410022D3E740C022D3E740502B5
:102D19002D3E7407022D3E7409022D3E740A022DC0
:102D29003E740B022D3E740D022D3E740E022D3E93
:102D3900740F022D3E90004D128B6D229001781276
:0E2D49002CBC9006D0122D02900178E06004A0
:102D5700122DDD2290684305A29000527B10128B42
:102D67003422900178E0B48003022D7B50FB122DB2
:102D7700A0022D7E128E3B90018FE0600122900110
:102D870083E0F490019AF0900182E0F4900199F0C9
:102D97009006D0E09006D1F022900178E070139071
:102DA700019AE0F4900183F0900199E0F490018298
:102DB700F022900178122DC9900183F0900182EFE3
:102DC700F022E075F002A41414FB90729B93FFEBC2
:102DD7000490729B9322122E8A900182122DF01278
:102DE7002E91900183122E12227408C39FFBE005D7
:102DF700A290005223FAA2E0122E43F0A3EADFF4D6
:102E0700EB7001227420F0A3DBFA22EF700C7B0831
:102E170090005A7420F0A3DBFA227408C39FFBE0EA
:102E270005A290005A23FAA2E0122E43F0A3EADF8C
:102E3700F4EB7001227420F0A3DBFA22400374A59F
:102E47002274FF22900178E070099006D1E0900685
:102E5700D0F022B48006C3947F022E6550F8122E5C
:102E67006D9006D0F022B4200374012240FBB43FDA
:102E77000374022240FBC3944075F00884240312B4
:102E87000A8A229006D0122E98229006D0122EC0BF
:102E970022E01475F003A4902EA2737F08227F0806
:102EA700227F05227F07227F08227F08227F0822B0
:102EB7007F08227F08227F0822E01475F003A49080
:102EC7002ECA737F08227F04227F00227F00227F81
:102ED70001227F02227F03227F05227F06227F07AE
:102EE7002220020122C205900179E004120CAEF003
:102EF700C202D24A2220030122C205900179E014BE
:102F0700120CAEF0C203D24A22900179E014B41039
:102F1700057460022F2350F990714993900186F050
:102F270022122F10900179E01475F006A4902F3823
:102F370073907039022FF8907049022FF8907059EA
:102F4700022FF8907069022FF8907079022FF8908D
:102F57007089022FF8907099022FF89070A9022FAC
:102F6700F89070B9022FF89070C9022FF89070D9B5
:102F7700022FF89070E9022FF89070F9022FF8905D
:102F87007109022FF8907119022FF8907129022FF9
:102F9700F8907139022FF8907149022FF890715902
:102FA700022FF8907169022FF8907179022FF8902B
:102FB7007189022FF8907199022FF89071A9022F49
:102FC700F89071B9022FF89071C9022FF89071D952
:102FD700022FF89071E9022FF89071F9022FF890FB
:102FE7007209022FF8907219022FF8907229022F96
:102FF700F805A29000527B10128B34222002012286
:10300700C205900175E004120BE7F0C202D232222A
:1030170020030122C205900175E014120BE7F0C2EC
:1030270003D23222900175E01460061475F0038410
:103037000475F006A490304073906DC90230589023
:103047006DD9023063906DE9023063906DF90230FB
:103057006305A29000527B10128B342205A29000C8
:10306700527B0F128B34900175E0147001221230DD
:103077007F900061128B6922900175E01470037ACA
:103087000022B4040302309950037A0122B40700E6
:103097005006C394037A0222C394067A03222002BD
:1030A7000122C205900176E004120CC1F0C202D2DF
:1030B700322220030122C205900176E014120CC1CE
:0E30C700F0C203D232229067CA05A2900052D6
:1030D5007B07128B34900176E0900059128B699032
:1030E5006E1105A290005A7B08128B342220020132
:1030F50022C205900177E004120C0DF0C2022220D5
:10310500030122C205900177E014120C0DF0C203F1
:1031150022900177E0FA747FC39AB47F0302313AB3
:10312500906E2905A29000527B0D128B34EA900017
:103135005F128B8222906DC905A29000527B1012FE
:103145008B342220020122C20590017AE004120C80
:10315500D4F0C2022220030122C20590017AE014B4
:10316500120CD4F0C2032290017AE0B408041231A3
:10317500912240FAB4090690716A0231ACB40A068C
:1031850090717A0231AC90718A0231AC90715A0516
:10319500A29000527B0F128B3490017AE09000616F
:1031A500128B691231DC2205A29000527B10128B22
:1031B500342290017AE0B408040231DC2240FAB4EA
:1031C50009061266A40231E0B40A0612669A0231B3
:1031D500E01266AE0231E090017AE014F9900179CF
:1031E500E01475F008A4299071DA93900187F02214
:1031F50020020122C20590017BE004120C1DF0C2E1
:10320500022220030122C20590017BE014120C1D4D
:10321500F0C2032290017BE014B4100302329950EE
:10322500FB75F006A490322E73906F2902328E90B2
:103235006F3902328E906F4902328E906F59023289
:103245008E906F6902328E906F7902328E906F89FF
:1032550002328E906F9902328E906FA902328E9053
:103265006FB902328E906FC902328E906FD90232D9
:103275008E906FE902328E906FF902328E9070094E
:1032850002328E90701902328E05A29000527B1088
:10329500128B3422C3940FFA7480C39AFA90702962
:1032A50005A29000527B0D128B34EA90005F128BC1
:1032B500822220020122C20590017CE004120C69E1
:1032C500F0C2022220030122C20590017CE0141203
:1032D5000C69F0C2032290017CE01475F006A490FD
:1032E50032E873906E390232F4906E490232F40579
:1032F500A29000527B10128B342220020122C205BB
:1033050090017DE004120C7CF0C202222003012210
:10331500C20590017DE014120C7CF0C203229001DD
:103325007DE01475F006A490333073906DC90233B7
:1033350042906E59023342906E6902334205A29063
:1033450000527B10128B342220020122C20590010B
:103355007EE004120C43F0C202C2B6222003012211
:10336500C20590017EE014120C43F0C203C2B622DE
:1033750090017EE01475F006A490338273906EB9C7
:10338500023394906EC9023394906ED9023394053A
:10339500A29000527B10128B342220020122C2051A
:1033A50090017FE004120C56F0C202222003012294
:1033B500C20590017FE014120C56F0C20322900161
:1033C5007FE01475F006A49033D073906EE9023354
:1033D500D9906EF905A29000527B10128B34229081
:1033E5000166E0B4090122B40A0122E56B30E52447
:1033F500203C0122D232C23C900166E0B4083290F2
:1034050006A3124BEFE56C04F09006AF124BEFE507
:103415006F04F022D23C1234DB12355112343A904B
:103425000201E07003856C6D9004B6E07003856F52
:103435006E22302F2290726A05A29000527B0912EB
:0E3445008B34123460900166E0B40304123B35
:103453002F22B40403123B2F221234D122E56C1223
:10346300349905A290005B7B02128B349067CA05E6
:10347300A290005D7B01128B34E56F12349905A293
:1034830090005E7B02128B349067CA05A2900060A5
:103493007B02128B342275F004A49034A1739072D2
:1034A30073229072752290727722907279229072B1
:1034B3007B2290727D2290727F2290728122907281
:1034C30083229072852290728722907289225350B0
:1034D300FF4350DE4351D722E56B20E10574000220
:1034E300354820E205740102354820E305740202E1
:1034F300354820E4057406023548E56A20E0057482
:103503000302354820E105740402354820E20574BE
:103513000502354820E305740702354820E40574A5
:103523000802354820E505740902354820E605748C
:103533000A02354820E705740B023548205403E599
:103543006C22E56F22205403F56C22F56F2275F08F
:103553000AA4903559735350FD4350DC4351D7228D
:103563005350FB4350DA4351D7225350F74350D6BD
:103573004351D7225350EF4350CE4351D722535098
:10358300BF43509E4351D72253507F43505E435114
:10359300D7225351FE4351D64350DE225351FD43AC
:1035A30051D54350DE225351FB4351D34350DE22C6
:1035B3005351EF4351C74350DE225351BF435197F9
:1035C3004350DE2253517F4351574350DE222002A2
:1035D3000122C205900169E004120B29F0900168F1
:1035E300F0C2022220030122C205900169E01412F5
:1035F3000B29F0900168F0C20322E56B20E501225C
:10360300D2541287E512371F1236CA300807123513
:10361300D11235E722900169E0B4010A123726126C
:10362300373B12855222B4020A12389A1238AE126C
:10363300855222B4030A12391D12393112855222DE
:10364300B4040A12396A12397C12855222B4051F56
:103653001237571237701206A412098312092D125A
:1036630009549001727405F09001637401F022B45F
:10367300060A12385012386412855222B4070A120D
:1036830039951239A712855222B4080A123A421206
:103693003A5412855222B4090A123A6D123A7F1231
:1036A300855222B40A0A123A98123AAA1285522271
:1036B300B40B0A123AC3123AD512855222123AEEC9
:1036C300123B0212855222900169E0B401041237C1
:1036D3005022B402041238C222B403041239452220
:1036E300B4040412398E22B4050412378922B406B5
:1036F3000412389022B407041239B922B408041210
:103703003A6622B40904123A9122B40A04123ABC6A
:1037130022B40B04123AE722123B1622900169E00D
:10372300022B2920020122C20590018BE004120B17
:10373300C1F0C202129E182220030122C205900189
:103743008BE014120BC1F0C203129E182290018B5E
:10375300E0022BCE20020122C20590018FE0F90482
:10376300120CA2F0C2021238201237AD222003013C
:1037730022C20590018FE0F914120CA2F0C20312C9
:1037830038201237AD2290018F122CBC9006D11233
:103793002D0290018FE0600412380D2290685305CA
:1037A300A29000527B10128B342290018FE0B480E0
:1037B300030237BF50FB1237E40237C2128E4E901A
:0E37C3000178E060012290019AE0F490018309
:1037D100F0900199E0F4900182F09006D1E090061A
:1037E100D0F02290018FE07013900183E0F49001FA
:1037F1009AF0900182E0F4900199F02290018F12E9
:103801002DC990019AF0900199EFF022123842905F
:103811000199122DF012384990019A122E1222901C
:10382100018FE070099006D0E09006D1F022B480BB
:1038310006C3947F02383A50F8122E6D9006D1F0EB
:10384100229006D1122E98229006D1122EC022204B
:10385100020122C205900190E004120CAEF0C202F6
:10386100D24B2220030122C205900190E014120CD8
:10387100AEF0C203D24B22900190E014B410057453
:103881006002388B50F99071499390019DF022129A
:103891003878900190E0022F2F20020122C205907A
:1038A100018CE004120BE7F0C202D23222200301A4
:1038B10022C20590018CE014120BE7F0C203D23250
:1038C1002290018CE01460061475F003840475F0F5
:1038D10006A49038D773906DC90238EF906DD90264
:1038E10038FA906DE90238FA906DF90238FA05A2BA
:1038F1009000527B10128B342205A29000527B0F54
:10390100128B3490018CE014700122123916900050
:1039110061128B692290018CE00230832002012226
:10392100C20590018DE004120CC1F0C202D2322214
:1039310020030122C20590018DE014120CC1F0C2D6
:1039410003D232229067CA05A29000527B07128BE4
:103951003490018DE0900059128B69906E1105A28F
:1039610090005A7B08128B342220020122C205905A
:10397100018EE004120C0DF0C2022220030122C2CA
:103981000590018EE014120C0DF0C2032290018EFD
:10399100E002311A20020122C205900191E00412D5
:1039A1000CD4F0C2022220030122C205900191E051
:1039B10014120CD4F0C20322900191E0B408041255
:1039C10039DE2240FAB4090690716A0239F9B40A63
:1039D1000690717A0239F990718A0239F990715A17
:1039E10005A29000527B0F128B34900191E0900060
:1039F10061128B69123A292205A29000527B1012A2
:103A01008B3422900191E0B40804023A292240FA51
:103A1100B409061266A4023A2DB40A0612669A0285
:103A21003A2D1266AE023A2D900191E014F99001FF
:103A310090E01475F008A4299071DA9390019EF03A
:103A41002220020122C205900192E004120C1DF015
:103A5100C2022220030122C205900192E014120C3D
:103A61001DF0C20322900192E002321D20020122C8
:103A7100C205900193E004120C69F0C202222003F6
:103A81000122C205900193E014120C69F0C20322D5
:103A9100900193E00232DF20020122C205900194DD
:103AA100E004120C7CF0C2022220030122C2059024
:103AB1000194E014120C7CF0C20322900194E00204
:103AC100332720020122C205900195E004120C4324
:103AD100F0C2022220030122C205900195E01412D6
:103AE1000C43F0C20322900195E0023379200201D8
:103AF10022C205900196E004120C56F0C202C2B532
:103B01002220030122C205900196E014120C56F006
:103B1100C203C2B522900196E01475F006A4903B51
:103B21002373906F090233D9906F190233D99067CB
:103B3100CA05A290004B7B04128B3422E56B20E571
:0E3B41000122123B50123B86123BBC12297926
:103B4F002220020122C205305310900180E004129E
:103B5F000CFAF0900197F0023B8120540C900180F9
:103B6F00E004120CFAF0023B81900197E004120C72
:103B7F00FAF0C202D2362220030122C205305310BE
:103B8F00900180E014120CFAF0900197F0023BB70D
:103B9F0020540C900180E014120CFAF0023BB79005
:103BAF000197E014120CFAF0C203D23622205413FC
:103BBF00900180123BFA123B2F900180123D1D1293
:103BCF008D9222900197123BFA123B2F9001971280
:103BDF003D1D128DA522900180123BFA123B2F90B2
:103BEF000180123D1D128D92023BD2E0B42B069044
:103BFF00774C023D0C50F81475F006A4903C0F73EF
:103C0F009074AC023D089074BC023D089074CC02D5
:103C1F003D089074DC023D089074EC023D089074EE
:103C2F00FC023D0890750C023D0890751C023D0882
:103C3F0090752C023D0890753C023D0890754C0222
:103C4F003D0890755C023D0890756C023D089075BB
:103C5F007C023D0890758C023D0890759C023D08D2
:103C6F009075AC023D089075BC023D089075CC0272
:103C7F003D089075DC023D089075EC023D0890758B
:103C8F00FC023D0890760C023D0890761C023D0820
:103C9F0090762C023D0890763C023D0890764C02BF
:103CAF003D0890765C023D0890766C023D08907658
:103CBF007C023D0890768C023D0890769C023D0870
:103CCF009076AC023D089076BC023D089076CC020F
:103CDF003D089076DC023D089076EC023D08907628
:103CEF00FC023D0890770C023D0890771C023D08BE
:103CFF0090772C023D0890773C123F682205A290E6
:103D0F0000527B10128B3490004F7455F022E0B4A8
:103D1F002B03023D2D50FB900050128B6D22C3944C
:103D2F002A900050128B6D22E56B20E50122123D87
:103D3F004A123D80123DB61229792220020122C279
:103D4F0005305310900181E004120D0DF090019891
:103D5F00F0023D7B20540C900181E004120D0DF018
:103D6F00023D7B900198E004120D0DF0C202D23794
:103D7F002220030122C205305310900181E014125A
:103D8F000D0DF0900198F0023DB120540C9001817F
:103D9F00E014120D0DF0023DB1900198E014120DD8
:103DAF000DF0C203D23722205413900181123DF43B
:103DBF00123B2F900181123F79128DB822900198FA
:103DCF00123DF4123B2F900198123F79128DCB22A6
:103DDF00900181123DF4123B2F900181123F791215
:103DEF008DB8023DCCE0B43707907D79123D0C229F
:103DFF0050F7B42B03023E09400BC3942B75F0060A
:103E0F00A4903F19731475F006A4903E1D73907A19
:103E1F0019023F64907A29023F64907A39023F6415
:103E2F00907A49023F64907A59023F64907A69020E
:103E3F003F64907A79023F64907A89023F64907A66
:103E4F0099023F64907AA9023F64907AB9023F6465
:103E5F00907AC9023F64907AD9023F64907AE9025E
:103E6F003F64907AF9023F64907B09023F64907B34
:103E7F0019023F64907B29023F64907B39023F64B3
:103E8F00907B49023F64907B59023F64907B6902AB
:103E9F003F64907B79023F64907B89023F64907B03
:103EAF0099023F64907BA9023F64907BB9023F6403
:0E3EBF00907BC9023F64907BD9023F64907BE8
:103ECD00E9023F64907BF9023F64907C09023F64F4
:103EDD00907C19023F64907C29023F64907C3902EA
:103EED003F64907C49023F64907C59023F64907C12
:103EFD0069023F64907C79023F64907C89023F6443
:103F0D00907C99023F64907CA9023F64907CB90239
:103F1D003F64907CC9023F64907CD9023F64907CE1
:103F2D00E9023F64907CF9023F64907D09023F6491
:103F3D00907D19023F64907D29023F64907D390286
:103F4D003F64907D49023F64907D59023F64907DAE
:103F5D0069023F64907D79123F682205A29000525C
:103F6D007B10128B3490004F7450F022E0B4370365
:103F7D00023F8950FB900050128B6D22C3943690F6
:103F8D000050128B6D2220020122C20590016CE0BF
:103F9D0004120B4FF0C2022220030122C205900130
:103FAD006CE014120B4FF0C20322E56B20E50122E9
:103FBD001285521287E512401C123FFF300807127E
:103FCD003F93123FA52290016CE0B4010A305006D8
:103FDD0012404F12406122B402071240AF1240C48A
:103FED0022B40307124110124122221241581241EC
:103FFD006A2290016CE0B4010412407322B40204F1
:10400D001240E622B403041241342212417C229064
:10401D00016CE01475F006A490402973906AD902E2
:10402D004041906AE3024041906AED024041906A3E
:10403D00F7024041122B9605A29000487B0A128B85
:10404D00342220020122C205900173E004120A44B9
:10405D00F0C2022220030122C205900173E0141266
:10406D000A44F0C203229001E7E0B4021A9067CA35
:10407D0005A29000527B0D128B34900173E0241435
:10408D0090005F128B82229067CA05A29000527B2E
:10409D000A128B34906B1505A290005C7B06128B77
:1040AD00342220020122C2059001E7E004120C30F7
:1040BD00F0C2021240D92220030122C2059001E76D
:1040CD00E014120C30F0C2031240D9229001E7E047
:1040DD00147003C25022D250229001E7E01475F003
:1040ED0006A49040F373906B15024105906B250269
:1040FD004105906B3502410505A29000527B1012CF
:10410D008B342220020122C205D25A9001E8E0D25E
:10411D00E2F0C2022220030122C205C25A9001E838
:10412D00E0C2E2F0C203229067CA05A29000527B62
:10413D000A128B34205A06906B4502414D906B4B01
:10414D0005A290005C7B06128B342220020122C254
:10415D00059001E6E004120B62F0C2022220030179
:10416D0022C2059001E6E014120B62F0C203229008
:10417D0067CA05A29000527B0A128B349001E6E0CB
:10418D001475F006A490419673906B510241A59061
:10419D006B450241A5906B4B05A290005C7B06120E
:1041AD008B342220020122C20590016DE004120B16
:1041BD009BF0C2022220030122C20590016DE01482
:1041CD00120B9BF0C20322E56B20E50122128552F2
:1041DD001287E512422512420F3008071241B01224
:1041ED0041C22290016DE0B4010712427F1242914B
:1041FD0022B40207124412124424221245A512457C
:10420D00B72290016DE0B401041242A322B402045E
:10421D00124436221245C92290016DE01475F00644
:10422D00A490423273906B57024244906B610242EC
:0E423D0044906B6B024244122B9605A2900037
:10424B00487B0A128B342230082205A290016DE0C4
:10425B00B4010B9001E3E09006CDF0024274B4027E
:10426B00089001E4E09006CEF005A2222005012281
:10427B009067EA2220020122C2059001E3E00412BA
:10428B000BD4F0C2022220030122C2059001E3E00D
:10429B0014120BD4F0C203229001E3E01475F00664
:1042AB00A49042B073906BB702437C906BC20243F5
:1042BB007C906BCD02437C906BD802437C906BE37C
:1042CB0002437C906BEE02437C906BF902437C9033
:1042DB006C0402437C906C0F02437C906C1A02437B
:1042EB007C906BCD02439A906BD802439A906BE310
:1042FB0002439A906BEE02439A906BF902439A90A9
:10430B006C0402439A906BCD0243B8906BD8024376
:10431B00B8906BE30243B8906BEE0243B8906BF925
:10432B000243B8906C040243B8906BCD0243D69015
:10433B006BD80243D6906BE30243D6906BEE0243ED
:10434B00D6906BF90243D6906C040243D6906BCD9A
:10435B000243F4906BD80243F4906BE30243F49066
:10436B006BEE0243F4906BF90243F4906C0402433E
:10437B00F412425205A29000577B0B128B34906BB8
:10438B008512425205A29000527B05128B342212E9
:10439B00425205A29000577B0B128B34906B8A1202
:1043AB00425205A29000527B05128B3422124252CC
:1043BB0005A29000577B0B128B34906B8F124252DD
:1043CB0005A29000527B05128B342212425205A299
:1043DB009000577B0B128B34906B9412425205A2B8
:1043EB009000527B05128B342212425205A2900090
:1043FB00577B0B128B34906B9912425205A2900093
:10440B00527B05128B342220020122C2059001E45B
:10441B00E004120BD4F0C2022220030122C2059049
:10442B0001E4E014120BD4F0C203229001E4E01477
:10443B0075F006A490444373906BB702450F906BD5
:10444B00C202450F906BCD02450F906BD802450F02
:10445B00906BE302450F906BEE02450F906BF902E8
:10446B00450F906C0402450F906C0F02450F906C3A
:10447B001A02450F906BCD02452D906BD802452D3E
:10448B00906BE302452D906BEE02452D906BF9027C
:10449B00452D906C0402452D906BCD02454B906BD6
:1044AB00D802454B906BE302454B906BEE02454BAC
:1044BB00906BF902454B906C0402454B906BCD020F
:1044CB004569906BD8024569906BE3024569906B27
:1044DB00EE024569906BF9024569906C04024569DF
:1044EB00906BCD024587906BD8024587906BE302AA
:1044FB004587906BEE024587906BF9024587906C70
:10450B000402458712425205A29000577B0B128B77
:10451B0034906B9E12425205A29000527B05128B77
:10452B00342212425205A29000577B0B128B34900F
:10453B006BA312425205A29000527B05128B3422C0
:10454B0012425205A29000577B0B128B34906BA832
:10455B0012425205A29000527B05128B342212425A
:10456B005205A29000577B0B128B34906BAD12420D
:10457B005205A29000527B05128B34221242520537
:10458B00A29000577B0B128B34906BB212425205E8
:10459B00A29000527B05128B342220020122C2050D
:1045AB00900171E004120BAEF0C202222003012233
:0E45BB00C205900171E014120BAEF0C2032293
:1045C900906B7505A29000527B0E128B349001718D
:1045D900E014900060128B69906B8405A2900061D1
:1045E9007B01128B341245F222300E0122900171A7
:1045F900E01475F00CA4120603C2AD8582448583CC
:1046090045858246858347D2AD900171E01475F0E6
:104619000CA412061BC2AD85824885834985824A4E
:1046290085834B85824C85834D85824E85834FD208
:10463900AD22900167E0F9124646E9F022E56B44A4
:10464900E1F47006E56AF470152230E1037901227C
:1046590030E2012230E30379022230E40122E56AE3
:10466900F430E0012230E10379032230E2037904D6
:104679002230E30379052230E4012230E50379068B
:104689002230E60379082230E70379072222C0E0C5
:104699008582378583387837900167E014F53B7553
:1046A9003C00793B1203868682088683D0E02290FB
:1046B9000167E0900047128B699000487420F0224E
:1046C90020020122C20590016EE004120B3CF0C2E7
:1046D900022220030122C20590016EE014120B3C54
:1046E900F0C20322E56B20E6012220E501221246F1
:1046F9003B1246B812474212472C3008071246C9E6
:104709001246DB2290016EE0B4010712477D124781
:104719009922B40207124951124969221249E61233
:1047290049FB2290016EE0B401041247E322B4026E
:104739000412498122124A102290016EE01475F088
:1047490006A490474F73906A6902476F906A740292
:104759004761906A7E024761122B9605A290004933
:104769007B09128B3422122B9605A29000487B05F7
:10477900128B342220020122C2059001A21246970F
:10478900E0F904120CA2F0C2021247B5124819222C
:1047990020030122C2059001A2124697E0F91412E2
:1047A9000CA2F0C2031247B5124819229001A212B5
:1047B9004697E0700F9006D21248A9E09006D212EF
:1047C9004697F022B48006C3947F0247D850F81266
:1047D9002E6D9006D2124697F0229001A2124697AA
:1047E900122CBC9006D2124697122D029001A212E9
:1047F9004697E060041249242290686305A290005C
:10480900527B0F128B341248ED900061128B692292
:104819009001A2124697E0B4800302482E50FB1281
:104829004868024831128E619001A21248A9E060DD
:1048390001229001D41248FFE0F49001D41248C932
:10484900F09001D31248FFE0F49001D31248C9F067
:104859009006D2124697E09006D21248A9F022900B
:1048690001A2124697E0701F9001D41248C9E0F4E2
:104879009001D41248FFF09001D31248C9E0F49096
:1048890001D31248FFF0229001A2124697122DC9B6
:104899009001D41248FFF09001D31248FFEFF022A3
:1048A900C0E085823785833878371248ED14F53BA7
:1048B900753C00793B1203868682088683D0E02204
:1048C900C0E085823785833878371248ED1475F052
:1048D90002A4F53B753C00793B1203868682088663
:1048E90083D0E022900167E0B40506C3940402482E
:1048F900FE50F8240422C0E0858237858338783752
:10490900900167E01475F002A4F53B753C00793B12
:104919001203868682088683D0E02212493D9001DF
:10492900D31248FF122DF01249479001D41248FFC3
:0E493900122E12229006D2124697122E9822AB
:104947009006D2124697122EC02220020122C205DB
:104957009001AA124697E004120CAEF0C202124967
:10496700AD2220030122C2059001AA124697E01446
:10497700120CAEF0C2031249AD2212498F9001AA60
:10498700124697E0122F2F229001AA124697E014A1
:10499700B4100574600249A550F9907149939001CC
:1049A700BA124697F022900167E01475F005A490BB
:1049B70049BA7379010249DF79020249DF790402B2
:1049C70049DF79080249DF79100249DF7920024976
:1049D700DF79400249DF79809001C2E049F0222067
:1049E700020122C2059001C3124697E004120CD4BB
:1049F700F0C2022220030122C2059001C31246978A
:104A0700E014120CD4F0C203229001C3124697E0BF
:104A1700B40804124A382240FAB4090690716A02AF
:104A27004A56B40A0690717A024A5690718A024A27
:104A37005690715A05A29000527B0F128B34900149
:104A4700C3124697E0900061128B69124A892205CA
:104A5700A29000527B10128B34229001C31246970A
:104A6700E0B40804024A892240FAB409061266A48F
:104A7700024A90B40A0612669A024A901266AE0279
:104A87004A909001C3124697E014FF9001AA12467C
:104A970097E01475F008A42F9071DA939001CB1268
:104AA7004697F02220580122C258124B014350DE8C
:104AB7004351D7E550C2E0F550D23AD23AD23B1231
:104AC7004B16128522125713124B3512853A125E76
:104AD700D1C232124ADE22900170E0B4010990027D
:104AE7000E128670028564B402099004C312869977
:104AF7000285644350DE4351D7229006A3124BEF41
:104B0700E014F56C9006AF124BEFE014F56F2290AE
:104B1700068B124BEFE0B43A08900180F01290AF89
:104B27002240F6C3943A900181F01294D322900662
:104B370097124BEFE0B43A08900197F01291642274
:104B470040F6C3943A900198F01294EB22E56B205B
:104B5700E50122900170E0B403012290016FE0F9B2
:104B6700124B6DE9F022E56B44E1F47008E56AF455
:104B77007028C2592220596FD25930E105790102B4
:104B87004BEB30E2057902024BEB30E30579030288
:104B97004BEB30E4057907024BEB20594AD259E534
:104BA7006AF430E0057904024BEB30E10579050240
:104BB7004BEB30E2057906024BEB30E3057908024F
:104BC7004BEB30E4057909024BEB30E505790A0236
:104BD7004BEB30E605790B024BEB30E705790C021E
:104BE7004BEB790CD2582222C0E085823785833877
:104BF700783790016FE014F53B753C00793B120361
:104C0700868682088683D0E02290016FE090004775
:104C1700128B6D2220020122C205900170E004125E
:104C27000B88F0C202124ADE2220030122C205903D
:104C37000170E014120B88F0C203124ADE22E56B02
:104C470020E50122E56B20E60122124B54124CB2FB
:104C5700124C90300807124C1B124C3022900170F6
:104C6700E0B4010C124CED124D04C254124ADE227C
:104C7700B4020C124D88124D9FD254124ADE2212F2
:104C87004DF3124E05124ADE22900170E0B4010A7C
:104C9700124C10124E2F124D1B22B4020A124C1046
:104CA700124E59124DB622124E1722900170E0147F
:0E4CB70075F006A4904CBF73906874024CD147
:104CC500906877024CD1906883024CDF122B9605D1
:104CD500A29000497B01128B3422122B9605A290DB
:104CE50000467B0C128B342220020122C20590065D
:104CF5008B124BEFE004120D20F0D258C202222095
:104D0500030122C20590068B124BEFE014120D2011
:104D1500F0D258C20322124D1F2290068B124BEF80
:104D2500E0B43A13123BFB90068B124BEF123D1D7C
:104D350090687B124D582240EBC3943A123DF59092
:104D4500068B124BEFE0C3943A123F7A90687D12BE
:104D55004D582205A290004E7B01128B342290689B
:104D65007905A29000487B02128B349006BCE09036
:104D7500004A128B6D9067CA05A290004C7B011208
:104D85008B342220020122C205900697124BEFE0D8
:104D950004120D20F0D258C2022220030122C205BE
:104DA500900697124BEFE014120D20F0D258C20373
:104DB50022124DBA22900697124BEFE0B43A131225
:104DC5003BFB900697124BEF123D1D90687B124DF1
:104DD500582240EBC3943A123DF5900697124BEFDB
:104DE500E0C3943A123F7A90687D124D5822200212
:104DF5000122C2059006BBE004120D6CF0C202222E
:104E050020030122C2059006BBE014120D6CF0C20E
:104E150003229067CA05A29000527B0E128B349034
:104E250006BBE0900060128B6D229067CA05A290C8
:104E3500004A7B01128B34E56C12349905A290006F
:104E45004B7B02128B349067CA05A290004D7B0103
:104E5500128B34229067CA05A290004A7B01128BFF
:104E650034E56F12349905A290004B7B02128B3406
:104E75009067CA05A290004D7B01128B3422200257
:104E85000122C205900172E004120B75F0C20222E4
:104E950020030122C205900172E014120B75F0C2C5
:104EA5000322303C01221285521287E5124F32123D
:104EB5004F01125108300807124E83124E95229069
:104EC5000172E01475F003A4904ED173024EE00216
:104ED5004EE5024EEC024EF3024EFAC202C2032226
:104EE500124FC7124FD922124FF6125008221250F4
:104EF50025125031221250D71250E322900160E062
:104F0500600122906A2105A29000527B10128B3419
:104F150022906A3105A29000527B10128B342290A8
:104F250067BA05A29000527B10128B342290017251
:104F3500E01475F006A4904F3F739069EF024F5D42
:104F45009069F9024F6B906A03024F7C906A0D02DB
:104F55004F8D906A17024FAA122B9605A290004812
:104F65007B0A128B3422122B9605A29000487B08EF
:104F7500128B34124FEB22122B9605A29000487B20
:104F850008128B3412501A22122B9605A290004853
:104F95007B05128B349006D0122D02745590004F6C
:104FA500F01250FD22122B9605A29000487B0512A7
:104FB5008B349006D1122D02745590004FF012508B
:104FC500FD2220020122C205900161E004120A7748
:104FD500F0C2022220030122C205900161E01412F1
:104FE5000A77F0C20322900161E0900050128B6DA8
:104FF5002220020122C205900162E004120A77F024
:10500500C2022220030122C205900162E014120AA5
:1050150077F0C20322900162E0900050128B6D225E
:1050250020020122C20512503DC2022220030122A4
:0E503500C205125044C203229006D012504B06
:10504300229006D012509122E01475F003A49050E0
:10505300557302507302507D0250870250870250ED
:105063008702508702508702508702508702508779
:10507300900163E004120A9DF022900163E00412A0
:105083000AB0F022900163E004120AC3F022E01494
:1050930075F003A490509B730250B90250C30250A1
:1050A300CD0250CD0250CD0250CD0250CD0250CD95
:1050B3000250CD0250CD900163E014120A9DF022FC
:1050C300900163E014120AB0F022900163E014121D
:1050D3000AC3F02220020122C2051250EFC20222AB
:1050E30020030122C2051250F6C203229006D112F8
:1050F300504B229006D112509122900163E0900010
:1051030050128B6D22E56B30E5089001E8E0C2E0B8
:10511300F0229001E8E020E043D2E0F0124F2412A5
:105123000375900172E0B40109128EAA128E9A02DD
:105133005156B40206125160025156B4030612517D
:105143006B025156B4040612527E02515612529209
:10515300025156124F169001607404F02220540439
:10516300125176221251B8222054041251FA2212FB
:10517300523C2290065305A2900201E0120A67FAFC
:105183009001E905A2F0A370057C010251A705A2D5
:10519300E0C3940CC3956CA305A2F0A3DAF09002CC
:1051A30001E004FC900161128F5205A2ECFB900612
:1051B30053128D5E2290066005A29004B6E0120A97
:1051C30067FA90049E05A2F0A370057C010251E9E1
:1051D30005A2E0C3940CC3956FA305A2F0A3DAF074
:1051E3009004B6E004FC900161128F5205A2ECFB1F
:1051F300900660128D5E2290066D05A2900201E07A
:10520300120A67FA9001E905A2F0A370057C010276
:10521300522B05A2E0C3940CC3956CA305A2F0A383
:10522300DAF0900201E004FC900162128FC305A240
:10523300ECFB90066D128D5E2290067A05A2900417
:10524300B6E0120A67FA90049E05A2F0A370057CEB
:105253000102526D05A2E0C3940CC3956FA305A28E
:10526300F0A3DAF09004B6E004FC900162128FC35D
:1052730005A2ECFB90067A128D5E229006D0129066
:105283001112904305A27B02900182128D5E22903F
:1052930006D112901112904305A27B02900199123C
:1052A3008D5E221252B3E56B20E60122124B54228B
:1052B30090688F05A29000427B01128B3490016F9E
:1052C300E0900043128B6D9067CA05A29000457B66
:1052D30001128B34E56C12349905A29000467B02CF
:1052E300128B349067CA05A29000487B01128B345D
:1052F30012535A9067CA05A290004D7B01128B345A
:1053030012549490689F05A29000527B01128B3433
:105313009006BCE0900053128B6D9067CA05A29073
:1053230000557B01128B34E56F12349905A290006E
:10533300567B02128B349067CA05A29000587B01FA
:10534300128B341253939067CA05A290005D7B01C0
:10535300128B341254B32290068B124BEFE0B43A03
:10536300131253E290068B124BEF12542E90687B6C
:105373001253CC2240EBC3943A1253F590068B128E
:105383004BEFE0C3943A12544890687D1253CC22F9
:10539300900697124BEFE0B43A1312540890069715
:1053A300124BEF12546190687B1253D72240EBC328
:0E53B300943A12541B900697124BEFE0C394ED
:1053C1003A12547B90687D1253D72205A29000496E
:1053D1007B01128B342205A29000597B01128B3480
:1053E10022B42B0790004A7455F02250F790004ADE
:1053F1007450F022B4350790004A7455F02250F7EA
:1054010090004A7450F022B42B0790005A7455F062
:105411002250F790005A7450F022B4350790005A88
:105421007455F02250F790005A7450F022E0B42BDA
:105431000302543E50FB90004B128B6D22C3942A01
:1054410090004B128B6D22B4350302545750FB90E0
:10545100004B128B6D22C3943490004B128B6D2242
:10546100E0B42B0302547150FB90005B128B6D2250
:10547100C3942A90005B128B6D22B4350302548AC7
:1054810050FB90005B128B6D22C3943490005B1231
:105491008B6D223005041254D2229067CA05A29066
:1054A100004E7B01128B349006CBE090004F128BA3
:1054B10082223005041255B3229067CA05A29000DA
:1054C1005E7B01128B349006CCE090005F128B82E0
:1054D100229006CDE01475F006A49054DF73906815
:1054E100AF0255A89068B30255A89068B70255A8B5
:1054F1009068BB0255A89068BF0255A89068C30286
:1055010055A89068C70255A89068CB0255A8906825
:10551100CF0255A89068D30255A89068D70255A824
:105521009068DB0255A89068DF0255A89068E302F5
:1055310055A89068E70255A89068EB0255A89068B5
:10554100EF0255A89068F30255A89068F70255A894
:105551009068FB0255A89068FF0255A89069030264
:1055610055A89069070255A890690B0255A8906942
:105571000F0255A89069130255A89069170255A802
:1055810090691B0255A890691F0255A890692302D2
:1055910055A89069270255A890692B0255A89069D2
:1055A1002F0255A890693305A290004E7B04128BFF
:1055B10034229006CEE01475F006A49055C0739085
:1055C100693B02568990693F0256899069430256A8
:1055D1008990694702568990694B02568990694FB3
:1055E10002568990695302568990695702568990EB
:1055F100695B02568990695F025689906963025618
:105601008990696702568990696B02568990696F22
:10561100025689906973025689906977025689907A
:10562100697B02568990697F025689906983025687
:105631008990698702568990698B02568990698F92
:10564100025689906993025689906997025689900A
:10565100699B02568990699F0256899069A30256F7
:10566100899069A70256899069AB0256899069AF02
:105671000256899069B30256899069B7025689909A
:1056810069BB0256899069BF05A290005E7B041236
:105691008B342290029AE070037B002230560A90EC
:1056A100015CE060041265A622900174E0B4190661
:1056B1001257060256E690049CE0F57C90049BE0AC
:1056C10004B57C1590017DE0B402069001377400A9
:1056D100F090049B74000256DC50E9F090049BE0CA
:1056E10012591FE0FB90049DF012307F90015BF096
:1056F10090015CEAF090015FE0B2E0F01265B790D2
:10570100049DE0FB2290049CE012667B12591FE08D
:10571100FB2290029AE0700122128840900174E00D
:105721001475F003A490572A730257750258110299
:0E57310058640258930258EA02593A0259721B
:10573F000259B70259FC025A13025AA7025AE80239
:10574F005B26025B6E025BAE025BE7025C01025CF2
:10575F001B025C38025CEA025D53025DDC025E02F2
:10576F00025E0C025E4E125779221257801257CDED
:10577F002290029AE0120D46FA7BFF7C0090029B6A
:10578F0005A290020E128654E0A30B30E7FA05A291
:10579F00EBF0A305A20CDAF0EC90049CF0FF229042
:1057AF00049CE090029B8582378583387837F53BE0
:1057BF00753C00793B12038686820886832290010E
:1057CF0076E0F57C157C7E01B40101221257E2D5FB
:1057DF007CFA22EE75F00CA4FD0E1257AEEFFB7C97
:1057EF000005A290029BE0A32D05A2F0A305A20C39
:1057FF00ECB4FF0590049CF022DBEB90049CE02CB2
:10580F00F02212577912581B1258342290049CE040
:10581F00FB90039B05A2EB1412591FE005A2F0A306
:10582F0005A2DBF22290049CE0FB90029B05A29064
:10583F00039BE0A305A2F0A305A2DBF62290049C34
:10584F00E0FB90039B05A290029BE0A305A2F0A3AF
:10585F0005A2DBF62212577912581B12586E2290AE
:10586F00049CE0FC1414FBEC12591F05A290039C3E
:10587F007C00E0A305A2F0A305A20CDBF590049C2D
:10588F00E02CF02212577990049CE0B402012240E0
:10589F00FD12581B1258AA1258342290049CE0FC97
:1058AF001414FBEC1258CF05A290029C7C00E0A3CD
:1058BF0005A2F0A305A20CDBF590049CE02CF022CE
:1058CF0090039B8582378583387837F53B753C008D
:1058DF00793B1203868682088683221257799004B9
:1058EF009CE0B402012240FD12581B1258FE229078
:1058FF00049CE0FB12591F05A290039BE0A305A295
:10590F00F0A305A2DBF690049CE075F002A4F02250
:10591F0090029B8582378583387837F53B753C003D
:10592F00793B120386868208868322125779900468
:10593F009CE0B402012240FD12581B12595112581B
:10594F00342290049CE0FB1258CF05A290029BE0FA
:10595F00A305A2F0A305A2DBF690049CE075F0026C
:10596F00A4F02212577990049CE0B402012240FD6A
:10597F001259861258342290049CE0FB14FC7D00CF
:10598F0090029B05A290039B05A2ED12591F0DE0FB
:10599F0005A2F0A305A2EC12591F1CE005A2F0A36B
:1059AF001BEB700122DBE12212577990049CE0B4CB
:1059BF0002012240FD1259CB1258342290049CE070
:1059CF00FB14FC7D0090029B05A290039B05A2ECAB
:1059DF0012591F1CE005A2F0A305A2ED12591F0DCD
:1059EF00E005A2F0A31BEB700122DBE12212577935
:1059FF0090049CE0B402012240FD125986125A66AF
:105A0F001258342212577990049CE0B402012240BC
:105A1F00FD1259CB125A2A1258342290049CE0FEE0
:105A2F00FB14FC7D0090029B05A2125AA205A2ED69
:105A3F0012591F0DE005A2F00EA305A2EC12591F7B
:105A4F001CE005A2F00EA31BEB7004025A6022DBD0
:105A5F00DC90049CEEF02290049CE0FEFB14FC7D95
:105A6F000090029B05A2125AA205A2EC12591F1C0C
:105A7F00E005A2F00EA305A2ED12591F0DE005A23D
:105A8F00F00EA31BEB7004025A9C22DBDC90049CEB
:105A9F00EEF022EB1258CF2212577990049CE0B40B
:0E5AAF0002012240FD125ABB1258342290040C
:105ABD009CE014FB7C007D0190029BE0FF05A29011
:105ACD00039BEFF00CA305A2ED12591F0DE005A2EB
:105ADD00F00CA3DBED90049CECF0221257799004AE
:105AED009CE0B402012240FD125AFC12583422905F
:105AFD00049CE014FB7C0090029BE0FF05A2900348
:105B0D009BEFF00CA305A2EB12591FE005A2F00CC0
:105B1D00A3DBEE90049CECF02212577990049CE0EC
:105B2D00B402012240FD12581B12586E125B401236
:105B3D0058342290049CE01414FB7C007D019002EB
:105B4D009BE0FF05A290039BEFF00CA305A2ED12C5
:105B5D00591F0DE005A2F00CA3DBED90049CECF0B9
:105B6D002212577990049CE0B402012240FD125894
:105B7D001B12586E125B40125B8B1258342290042C
:105B8D009CE075F00284FCFB90039B05A2EC12587F
:105B9D00CFE0FF05A2E0CFF0A305A2EFF0A3DBF16C
:105BAD002212577990049CE0B401012240FD125B52
:105BBD00C21258342290049CE0FB90039B05A290E6
:105BCD00029BE0A305A2F0A3240CF0A305A2DBF237
:105BDD0090049CE075F002A4F02212577990049C79
:105BED00E0B401012240FD12581B125834125BC261
:105BFD001258342212577990049CE0B401012240CE
:105C0D00FD12581B12586E125BC2125834221257D5
:105C1D007990049CE0B401012240FD12581B1258EA
:105C2D006E125BC2125B8B12583422125C5B9004B5
:105C3D009CE0B4020A12584C125CAA12583422404D
:105C4D00F4125C92125C65125CAA12583422900216
:105C5D009AE0120D3302578790049CE0FBFDFF7E06
:105C6D00007C0090039B05A290029BE0A305A2F08F
:105C7D00A305A20CDBF50EEDFBEE12591FDFEC9028
:105C8D00049CECF02290049CE0FB12591F05A2909D
:105C9D00029BE0A305A2F0A305A2DBF622900176FC
:105CAD00E014700122FF7D0090049C125CC59004ED
:105CBD009CE00D8DF0A4F022E0FCFB0DECFB8DF0D3
:105CCD00A41258CF05A290039BED75F00CA4FEE035
:105CDD002EA305A2F0A305A2DBEFDFDF22125C5B92
:105CED0090049CE0B4020A12584C125D1312583401
:105CFD002240F412581B125834125C92125C651239
:105D0D005D1312583422900176E014700122FF7D4C
:105D1D000090049C125D2E90049CE00D8DF0A4F07B
:105D2D0022E0FCFB0DECFB8DF0A41258CF05A290E8
:105D3D00039BEF75F00CA4FEE02EA305A2F0A305C6
:105D4D00A2DBEFDFDF2212578090049CE0B4020A41
:105D5D0012584C125CAA1258342240F4125D731280
:105D6D005CAA1258342290049CE0FB7C0090039BAB
:105D7D0005A290029BE0A305A2F00CA305A2DBF502
:105D8D0090049CE014FB90029CE0A305A2F00CA3F0
:105D9D0005A2DBF590029BE0240CA305A2F00CA359
:105DAD0005A290049CE01414FB90029DE0A305A2B3
:105DBD00F00CA305A2DBF57B0290029BE0240CA363
:105DCD0005A2F00CA305A2DBF390049CECF02212CB
:105DDD00578090049CE0B4020A12581B125D1312F6
:105DED0058342240F4125D7312583412581B125D50
:105DFD001312583422125E16125CAA125834221253
:105E0D005E16125CAA125E3522900201E07001222C
:105E1D0090049CF0FB90039B05A29001E9E0A30583
:0E5E2D00A2F0A305A2DBF62290049CE0FB90FD
:105E3B00029B05A2EB141258CFE005A2F0A305A21A
:105E4B00DBF2221257792290054FE070037B002280
:105E5B0030570A90015EE060041265D42290018BEA
:105E6B00E0B41906125EC4025EA4900651E0F57C04
:105E7B00900650E004B57C15900194E0B4020690B6
:105E8B00013A7400F09006507400025E9A50E9F0EB
:105E9B00900650E01260B9E0FB900652F0123916F2
:105EAB0090015DF090015EEAF090015FE0B2E1F0ED
:105EBB001265E5900652E0FB22900651E012667BDC
:105ECB001260B9E0FB2290054FE07001221288F2BC
:105EDB0090018BE01475F003A4905EE873025F33BE
:105EEB00025FC60260190260480260840260D4023D
:105EFB00610C0261510261960261AD02623C026269
:105F0B007D0262BB02630302632702636002637A52
:105F1B000263940263B10264630264A702653002F8
:105F2B0065560265600265A2125F3722125F3E1250
:105F3B005F8B2290054FE0120D46FA7BFF7C0090A1
:105F4B00055005A29004C3128662E0A30B30E7FA5A
:105F5B0005A2EBF0A305A20CDAF0EC900651F0FFD2
:105F6B0022900651E090055085823785833878372B
:105F7B00F53B753C00793B120386868208868322AB
:105F8B0090018DE0F57C157C7E01B4010122125F3E
:105F9B00A0D57CFA22EE75F00CA4FD0E125F6CEF0F
:105FAB00FB7C0005A2900550E0A32D05A2F0A305F4
:105FBB00A20CDBF4900651E02CF022125F37125F3B
:105FCB00D0125FE922900651E0FB90039B05A2EBF8
:105FDB00141260B9E005A2F0A305A2DBF222900631
:105FEB0051E0FB90055005A290039BE0A305A2F0A6
:105FFB00A305A2DBF622900651E0FB90039B05A2C2
:10600B00900550E0A305A2F0A305A2DBF622125FD8
:10601B0037125FD012602322900651E0FC1414FB60
:10602B00EC1260B905A290039C7C00E0A305A2F0E2
:10603B00A305A20CDBF5900651E02CF022125F3782
:10604B00900651E0B402012240FD125FD012605F56
:10605B00125FE922900651E0FC1414FBEC1258CFAE
:10606B0005A29005517C00E0A305A2F0A305A20CAC
:10607B00DBF5900651E02CF022125F37900651E0D1
:10608B00B402012240FD125FD0126098229006519B
:10609B00E0FB1260B905A290039BE0A305A2F0A35D
:1060AB0005A2DBF6900651E075F002A4F0229005F4
:1060BB00508582378583387837F53B753C00793BC3
:1060CB00120386868208868322125F37900651E080
:1060DB00B402012240FD125FD01260EB125FE92285
:1060EB00900651E0FB1258CF05A2900550E0A30596
:1060FB00A2F0A305A2DBF6900651E075F002A4F026
:10610B0022125F37900651E0B402012240FD12616A
:10611B0020125FE922900651E0FB14FC7D009005F4
:10612B005005A290039B05A2ED1260B90DE005A2EC
:10613B00F0A305A2EC1260B91CE005A2F0A31BEBC7
:10614B00700122DBE122125F37900651E0B40201AD
:10615B002240FD126165125FE922900651E0FB14AB
:10616B00FC7D0090055005A290039B05A2EC1260EC
:10617B00B91CE005A2F0A305A2ED1260B90DE00574
:10618B00A2F0A31BEB700122DBE122125F3790061A
:10619B0051E0B402012240FD126120126200125F35
:0E61AB00E922125F37900651E0B40201224053
:1061B900FD1261651261C4125FE922900651E0FE89
:1061C900FB14FC7D0090055005A2125AA205A2ED10
:1061D9001260B90DE005A2F00EA305A2EC1260B998
:1061E9001CE005A2F00EA31BEB70040261FA22DB8E
:1061F900DC900651EEF022900651E0FEFB14FC7D86
:106209000090055005A2125AA205A2EC1260B91C11
:10621900E005A2F00EA305A2ED1260B90DE005A2FA
:10622900F00EA31BEB700402623622DBDC900651F0
:10623900EEF022125F37900651E0B402012240FDD0
:10624900126250125FE922900651E014FB7C007D36
:1062590001900550E0FF05A290039BEFF00CA30508
:10626900A2ED1260B90DE005A2F00CA3DBED9006DA
:1062790051ECF022125F37900651E0B4020122403E
:10628900FD126291125FE922900651E014FB7C0035
:10629900900550E0FF05A290039BEFF00CA305A227
:1062A900EB1260B9E005A2F00CA3DBEE900651EC0D
:1062B900F022125F37900651E0B402012240FD122C
:1062C9005FD01260231262D5125FE922900651E075
:1062D9001414FB7C007D01900550E0FF05A290039A
:1062E9009BEFF00CA305A2ED1260B90DE005A2F039
:1062F9000CA3DBED900651ECF022125F37900651AA
:10630900E0B402012240FD125FD01260231262D56F
:10631900126320125FE922900651125B8E22125FEE
:1063290037900651E0B401012240FD12633B125F30
:10633900E922900651E0FB90039B05A2900550E0ED
:10634900A305A2F0A3240CF0A305A2DBF290065149
:10635900E075F002A4F022125F37900651E0B40113
:10636900012240FD125FD0125FE912633B125FE91F
:1063790022125F37900651E0B402012240FD125FFC
:10638900D012602312633B125FE922125F37900635
:1063990051E0B402012240FD125FD0126023126362
:1063A9003B126320125FE9221263D4900651E0B4D4
:1063B900020A126001126423125FE92240F4126496
:1063C9000B1263DE125CAA125FE92290054FE012FC
:1063D9000D33025F45900651E0FBFDFF7E007C0016
:1063E90090039B05A2900550E0A305A2F0A305A286
:1063F9000CDBF50EEDFBEE1260B9DFEC900651EC0B
:10640900F022900651E0FB1260B905A2900550E018
:10641900A305A2F0A305A2DBF62290018DE014707A
:106429000122FF7D0090065112643E900651E00D55
:106439008DF0A4F022E0FCFB0DECFB8DF0A41258CA
:10644900CF05A290039BED75F00CA4FEE02EA305E9
:10645900A2F0A305A2DBEFDFDF221263D49006517D
:10646900E0B4020A12600112648C125FE92240F45E
:10647900125FD0125FE912640B1263DE12648C1290
:106489005FE92290018DE014700122FF7D009006E2
:1064990051125D2E900651E00D8DF0A4F022125F8D
:1064A9003E900651E0B4020A126001126423125FA1
:1064B900E92240F41264C7126423125FE9229006AC
:1064C90051E0FB7C0090039B05A2900550E0A305D9
:1064D900A2F00CA305A2DBF5900651E014FB900590
:1064E90051E0A305A2F00CA305A2DBF5900550E04D
:1064F900240CA305A2F00CA305A2900651E01414E4
:10650900FB900552E0A305A2F00CA305A2DBF57BE5
:1065190002900550E0240CA305A2F00CA305A2DB10
:0E652900F3900651ECF022125F3E900651E016
:10653700B4020A125FD012648C125FE92240F4128F
:1065470064C7125FE9125FD012648C125FE92212EE
:10655700656A126423125FE92212656A12642312C4
:106567006589229004B6E0700122900651F0FB90F5
:10657700039B05A290049EE0A305A2F0A305A2DB5E
:10658700F622900651E0FB90055005A2EB14125835
:10659700CFE005A2F0A305A2DBF222125F3722901B
:1065A700049DE0FB90015BE014F0600122C25622DB
:1065B700BA0103D25622BA020720E00122D256229C
:1065C700BA030720E003D2562222C256229006526F
:1065D700E0FB90015DE014F0600122C25722BA018E
:1065E70003D25722BA020720E10122D25722BA0367
:1065F7000720E103D2572222C25722900072E004FB
:10660700B410027400F0900062A98229F582E0229A
:10661700900076E0FA900073E004B40F0274FFF084
:106627009066EF932A900076F0900075E004B4101E
:10663700027400F0F9900076E0FA900062E5822992
:10664700F582EAF022900076E0FA900074E004B454
:10665700110274FFF09066FE932A900076F012669E
:10666700302212660254016008126602541F246029
:1066770022747F22F974FF89F084F5F01266028490
:106687002212660275F020842212660275F03384A6
:1066970024012212660275F0208424012212660268
:1066A70075F03F8424012212660275F033842403B7
:1066B7002212660275F010842212660275F01F849A
:1066C7002212660275F02084F812660275F03F8484
:1066D7002822126602540175F00CA4221266027574
:1066E700F0558475F00CA422037F2C0C0105712151
:1066F70033E6FF0B576818BD09A60D004B5D26351D
:1067070085B196114093C8D3464C414D452041521F
:10671700504547474941544F52204D4F44554C45EA
:10672700204555524F205241434B2056455253491D
:106737004F4E202D20323031332056455253494F8A
:106747004E20312E303020286329627920616D7008
:10675700657265204620204C20204120204D2020B6
:106767004520204152504547474941544F52203216
:10677700303133202056455253494F4E20312E3069
:106787003220202020202028632932303133202056
:10679700202020496E697420616C6C20446174610B
:1067A700203F204F4B202020202020202020202069
:1067B7004E4F2020506C65617365207761697420A6
:1067C70021202020202020202020202020202020C1
:1067D70020202020202020202020202020202020B2
:1067E70020202020202020202020202020202020A2
:1067F7002020206F6666415250202020424153538B
:10680700202043484F5244205343414C45204D4993
:1068170044492020534554555020584F55543A2049
:106827004C4953542020534156452020504C415940
:106837004C49535420444154412020206D697272C1
:106847006F72656420536571426173736D6972720B
:106857006F72656420536571204172706D69727241
:106867006F7265642053657120582D313A41203A83
:106877004220543A633A733A4C495354202020201B
:1068870020204C656E6768744C31322023432063A7
:1068970050303120417365715430302020442073CB
:0E68A700553136203473657141706F72416E49
:1068B50074724173657141436C6B4164756F4174CA
:1068C500726941646F74416761745631323756722B
:1068D5006E643173657131436C6B3164756F3174FE
:1068E500726931646F7431676174327365713243F3
:1068F5006C6B3264756F3274726932646F743267AF
:1069050061743373657133436C6B3364756F3374C2
:10691500726933646F7433676174347365713443BA
:106925006C6B3464756F3474726934646F74346776
:106935006174546D706F42706F72426E74724273FF
:10694500657142436C6B4264756F4274726942644F
:106955006F74426761745631323756726E6435739F
:10696500657135436C6B3564756F35747269356463
:106975006F74356761743673657136436C6B366455
:10698500756F3674726936646F7436676174377300
:10699500657137436C6B3764756F3774726937642B
:1069A5006F74376761743873657138436C6B38641D
:1069B500756F3874726938646F74386761743E41F5
:1069C50020203E4220203E414220582D3120582D86
:1069D5003220582D3320582D3420582D3520582D50
:1069E5003620582D3720582D38202020416C6C2D0D
:1069F500446174613E43686F72643A5530313E5369
:106A050063616C653A553031413E534551313655D8
:106A15003031423E534551313655303150726573F0
:106A25007320204B45594E4F544520212020535467
:106A35004F52414745204F4B202120202020202028
:106A450020204D4F44454E4F5445524550454154E5
:106A5500202020202052414E47452020202020473D
:106A65004C494445205345513A3136503031202068
:106A7500202020434C4F434B2020202020204741FD
:106A85005445202056454C4F4349545920534551B0
:106A9500552D4D4F44454C4F4F502D524553455460
:106AA50020204F55542D47415445202020204F5537
:106AB500542D4356584F55543A312031363A536583
:106AC500715030314241535320202031363A5365BD
:106AD50071503031202020202054454D504F20202A
:106AE5002020202053594E435245435620434C4FB6
:106AF500434B53454E4420434C4F434B524543561D
:106B050020535953455853454E44205359534558DE
:106B150065787465726E204D696469436C6F636B4B
:106B250020202020696E7465726E20436C6F636B44
:106B350043686F7264205472696767657220496E95
:106B45006E6F726D616C202068616C662020206F0D
:106B5500666620555345522D3120494E20555345E3
:106B6500522D3220494E2054554E452D4D4F44450A
:106B75005365742043562D4F5554733A202B315687
:106B85004172703A20582D313A20582D323A20580A
:106B95002D333A20582D343A20426173733A582DDB
:106BA500353A20582D363A20582D373A20582D3869
:106BB5003A20202020202020474C494445204E4F94
:106BC5005445524550454154202020534551554583
:106BD5004E43452020434C4F434B20414C4C2020F5
:106BE500434C4F434B2044554F2020434C4F434B80
:106BF500205452492020434C4F434B20444F5420AE
:106C05002020202020204741544556454C4F203117
:106C15002E2E31323756454C4F20416363526E64F8
:0E6C250020202020555345522D3120202020C4
:106C3300555345522D32436C61737369633A202077
:106C4300202020207570436C61737369633A2020A0
:106C53002020646F776E436C61737369633A2020FD
:106C63007570646F776E436C61737369633A202048
:106C7300646F776E7570436F70793A2020202075AA
:106C8300702B646F776E436F70793A2020202064F5
:106C93006F776E2B757050696E67506F6E673A2011
:106CA30020202020757050696E67506F6E673A2000
:106CB3002020646F776E50696E67506F6E673A205D
:106CC3007570646F776E50696E67506F6E673A20A8
:106CD300646F776E757046697420526F6F743A20D3
:106CE30020202020757046697420526F6F743A20FB
:106CF3002020646F776E46697420526F6F743A2058
:106D03007570646F776E46697420526F6F743A20A2
:106D1300646F776E7570466974204F637461763A59
:106D2300202020207570466974204F637461763A81
:106D33002020646F776E466974204F637461763ADE
:106D43007570646F776E466974204F637461763A29
:106D5300646F776E7570536B69703A202020202022
:106D6300202020207570536B69703A20202020204A
:106D73002020646F776E496E76657273696F6E3A21
:106D8300202020207570496E76657273696F6E3AA4
:106D93002020646F776E4F7264657265643A2020B9
:106DA3002020202075704F7264657265643A20203C
:106DB3002020646F776E2020202020202020202098
:106DC30052616E646F6D202020202020202020201F
:106DD3002020206F66662020202020202020206590
:106DE3006163683A2031416C7465726E6174652029
:106DF3003173743A2031416C7465726E617465202D
:106E0300326E643A20312020202020202032206F4F
:106E1300637461766573202020206D6178696D61EC
:106E23006C3A20313238506F7274616D2E54696D33
:106E3300653A203132372020202073746570206238
:106E43007920737465702020202020202020636F18
:106E53006D62696E65642061742061727065676735
:106E6300696F20656E642061742073657175656E4A
:106E7300636520656E64696E7465726E436C6F63DF
:106E83006B2F4D494449547269676765722D496E8A
:106E93002020312F3136547269676765722D496E30
:106EA300205469636B73547269676765722D496E09
:106EB300205374657073202053657175656E636527
:106EC30028476174652920202052657365742070FA
:106ED3006572204261722020417270656767696F35
:106EE3002052657365744F75742D333A20205665AF
:106EF3006C6F636974794F75742D333A43686F729D
:106F030064206E6F74654F75742D343A2020566576
:106F13006C6F636974794F75742D343A43686F727B
:106F230064206E6F746520202020202066697273B0
:106F330074206E6F7465202020202020206C6173E4
:106F430074206E6F7465416363656E743A20656186
:106F5300636820326E64416363656E743A206561D1
:106F6300636820337468416363656E743A206561B6
:106F7300636820347468416363656E743A206561A5
:106F8300636820357468416363656E743A20656194
:106F9300636820367468416363656E743A20656183
:0E6FA300636820377468416363656E743A203A
:106FB1006561636820387468416363656E743A2063
:106FC100656163682039746852616E646F6D3A203F
:106FD1002020312E2E31323752616E646F6D3A208E
:106FE1002036342E2E31323752616E646F6D3A2065
:106FF1002037362E2E31323752616E646F6D3A2052
:107001002039352E2E31323752616E646F6D3A2040
:107011003131322E2E31323752616E646F6D3A202A
:1070210020666F726D756C61202020202020202049
:107031006669783A2031323731205469636B3A20DE
:10704100312F36342074726933205469636B733A7B
:1070510020202020312F333236205469636B733A5C
:1070610020202020312F313631325469636B733A3D
:107071002020202020312F3832345469636B733A39
:107081002020202020312F3434385469636B733A27
:107091002020202020312F3239365469636B733A16
:1070A100202020312062617232205469636B733A6F
:1070B100312F33322074726934205469636B733A0F
:1070C100312F31362074726938205469636B733AF9
:1070D10020312F382074726931365469636B733AE9
:1070E10020312F342074726933325469636B733ADF
:1070F10020312F322074726936345469636B733ACC
:1071010020312F312074726939205469636B733ACD
:10711100312F313620646F7431385469636B733A9F
:1071210020312F3820646F7433365469636B733A9E
:1071310020312F3420646F7437325469636B733A92
:1071410020312F3220646F740103060C1830600265
:1071510004081020400912244820202020206164C6
:1071610061707465643A20203361646170742E72B9
:10717100616E646F6D3A312D3561646170742E7288
:10718100616E646F6D3A312D3861646170742E7275
:10719100616E646F6D3A332D3820206669782072F4
:1071A100616E646F6D3A2034382020202061636362
:1071B100656E7420206C6F6E6720202020616363F0
:1071C100656E742073686F72742020202020202047
:1071D10020206669783A2039380101010101010155
:1071E1000201010102020303040101020303040479
:1071F10007010203050708090F0103070A0D11130F
:107201001E01070D141B21273C010D1B2835434F7F
:1072110078010101010202020301010102020303DB
:1072210005010102030405050901020406080A0B10
:10723100120104080C101417240108101820282F1B
:1072410048010203040506070C010305080A0D0F96
:107251001801050B10151B1F30010B15202B353F95
:10726100600110203040505FC04B45594E4F54458E
:107271003A202043234320442344204520462346EB
:1072810020472347204123412042234330206D6181
:107291006A6F72203720202020520000FFFF8000FB
:1072A10080808888AAAA0808141422225555EEEE77
:1072B100E38EE388C30CDB6F9999BABAAB5ADB6EE4
:1072C100DB6AADADD6D6AAD5A9A9ABABDADA9249BC
:1072D100BBBBAA9AAAD7CAE2A9A9FFF08000AAA0BB
:1072E100AD60A940AD502950AB502A50ABC0A2406F
:1072F100B2C0BEF09200B6A0A0A0249002A09A0055
:1073010089800920BBE0A990A9E0BAE0EAC09240D7
:10731100A280B2C0B6D0FEA0F8008000C000E0009C
:0E732100F000A800B000D000FE008000AA001E
:10732F00D800E000EC00F400D400FF808000AA80B9
:10733F00DB00ED00F700B680CA80FFC08000AA8096
:10734F008A80EA80A500B580F580FFE08000AAA0C2
:10735F00D280EAC0F540F780E740FFF88000AAA886
:10736F00DB60E770BDA0F7B0F9F0FFFC8000AAA8C2
:10737F00DB68FDF8EDD8FAB0D49CFFFE8000AAAA16
:10738F00E9DCEEECF5DABDDCFAB2030004070C041D
:10739F0000040709040004070B040004060B040093
:1073AF0004080B040002040704000405070400048A
:1073BF00070E030003060C040004070A040004066A
:1073CF000A030005070C0400020507040002050A62
:1073DF00030003070C0400030709040003070A0452
:1073EF000003060A040003080A040002030704004E
:1073FF00030507030003070E040003060904000337
:10740F00060A030004080C040004080A030002071C
:10741F000C040005070A0300050A0C020000000017
:10742F00020001000002000200000200030000023F
:10743F000004000002000500000200060000020028
:10744F000700000200080000020009000002000A05
:10745F00000002000B000002000C00000200000000
:10746F000002000100000200020000020003000001
:10747F0002000400000200050000020006000002E6
:10748F0000070000020008000002000900000200CF
:10749F000A000002000B000002000C000020202058
:1074AF0020202020202020204D616A6F7220202074
:1074BF002020202020204D616A6F7220362020204E
:1074CF002020202020204D616A6F7220372020203D
:1074DF00202020204D616A6F7220376235202020D6
:1074EF00202020204D616A6F722037233520202005
:1074FF0020202020202020206164642032202020A2
:10750F00202020202020202061646420342020208F
:10751F00202020202020202061646420392020207A
:10752F0020202044696D696E69736865642020208E
:10753F002020202020202020202020203720202025
:10754F0020202020202020202020376235202020BE
:10755F00202020202020202073757320342020200D
:10756F0020207375732034207375732032202020F0
:10757F0020202050656E7461746F6E696320202027
:10758F0020202020202020204D696E6F7220202087
:10759F002020202020204D696E6F72203620202061
:1075AF002020202020204D696E6F72203720202050
:1075BF002020204D696E6F722037206235202020E9
:1075CF002020204D696E6F72203720233520202018
:1075DF0020204D696E6F722061646420322020205C
:1075EF0020204D696E6F722061646420342020204A
:1075FF0020204D696E6F7220616464203920202035
:10760F002044696D696E6973686564203720202096
:10761F0020202068616C662064696D20372020204F
:10762F00202020204175676D656E746564202020D1
:10763F00202020202020202020372023352020200C
:10764F00202020202020202073757320322020201E
:10765F0020202020202037207375732034202020F5
:10766F00202020202020466F757274687320202000
:10767F00496E74657276616C2020302D3020202089
:10768F00496E74657276616C2020302D3120202078
:0E769F00496E74657276616C2020302D3220A9
:1076AD002020496E74657276616C2020302D332058
:1076BD002020496E74657276616C2020302D342047
:1076CD002020496E74657276616C2020302D352036
:1076DD002020496E74657276616C2020302D362025
:1076ED002020496E74657276616C2020302D372014
:1076FD002020496E74657276616C2020302D382003
:10770D002020496E74657276616C2020302D3920F1
:10771D002020496E74657276616C20302D313020D9
:10772D002020496E74657276616C20302D313120C8
:10773D002020496E74657276616C20302D313220B7
:10774D002020202020757365722063686F72640895
:10775D00000305070206080B0000000006000407E1
:10776D0008010500000000000005000307080100E6
:10777D00000000000000060003070A0409000000D5
:10778D00000000060003050A0607000000000000C7
:10779D00070004070B01050800000000000C0003A2
:1077AD00070A010204050608090B05000204070972
:1077BD0000000000000000070004070B0105080091
:1077CD0000000000070004080B01060A000000007D
:1077DD0000050005070A0200000000000000070078
:1077ED0004070A0205080000000000070004070A4C
:1077FD000306090000000000070003070B0206083E
:10780D000000000000050003070802000000000052
:10781D000000050005060A0100000000000000053B
:10782D000005070801000000000000000500050725
:10783D000A0100000000000000050003070A050012
:10784D00000000000000050005070A02000000000E
:10785D000000000500040709020000000000000000
:10786D00070004060A0205080000000000070003D7
:10787D00060A0104080000000000070004070A02C0
:10788D0006080000000000070004070902050B00B0
:10789D0000000000040004070900000000000000C3
:1078AD0000040004070B00000000000000000400AD
:1078BD0004060A0000000000000000070003070A8C
:1078CD000205080000000000040003070900000085
:1078DD000000000000040003070A00000000000083
:1078ED000000070003070B02050800000000000759
:1078FD000004070B02050900000000000700020646
:10790D000A0305090000000000070003070A01052E
:10791D00080000000000070004070B020609000024
:10792D00000000070004070A020509000000000717
:10793D000003070A02050800000000000700030607
:10794D000A010508000000000007000307090105F2
:10795D000B0000000000070003070B0105080000E5
:10796D000000000900030709020406080B000000CF
:10797D00080004070A0103060900000000070004BF
:10798D00060A0105090000000000070004070A02AD
:10799D0006090000000000050003070801000000B3
:1079AD0000000000050005070902000000000000AE
:1079BD00000500040709020000000000000005009A
:1079CD000305070A00000000000000050004060A78
:1079DD000200000000000000070004080A0105076E
:1079ED00000000000008000306090104070A00005A
:1079FD000000060004080A0206000000000000074F
:107A0D000004080B02060A000000000020202020C0
:0E7A1D0020202020416C67657269616E202078
:107A2B00202020202020204172616269616E20207D
:107A3B002020202042616C696E657369616E202085
:107A4B00202020426C756573206D616A6F72202057
:107A5B00202020426C756573206D696E6F7220203B
:107A6B00202020202042797A616E74696E65202077
:107A7B0020202020204368726F6D61746963202081
:107A8B00202020202020446961746F6E696320449C
:107A9B006F75626C65204861726D6F6E6963202033
:107AAB002020202020456E69676D6174696320205A
:107ABB00202020202020456779707469616E20207A
:107ACB00202020202048696E64757374616E2048F5
:107ADB00756E67617269616E206D616A6F722048A5
:107AEB00756E67617269616E206D696E6F724A6146
:107AFB0070616E3A2068697261796F7368694A6167
:107B0B0070616E3A697761746F796F7368694A61F6
:107B1B0070616E3A6B756D6F69796F7368694A61E5
:107B2B0070616E3A2020202020696E73656E4A6169
:107B3B0070616E3A2020202020796F73656E4A6148
:107B4B0070616E3A2020726974737573656E4A6149
:107B5B0070616E3A2020202072796F73656E202041
:107B6B00206D616A6F72204C6F637269616E2020A9
:107B7B00207375706572204C6F637269616E202083
:107B8B0020204C796469616E206D696E6F722020C4
:107B9B002020202020202020204D616A6F72202081
:107BAB00202020202020204D616A6F72203620205B
:107BBB00202020202020204D616A6F72203720204A
:107BCB00202020204D616A6F7220372062352020E3
:107BDB002020202020202020204D696E6F72202035
:107BEB00202020202020204D696E6F72203620200F
:107BFB00202020202020204D696E6F7220372020FE
:107C0B004D696E6F72206861726D6F6E69634D6F37
:107C1B0064653A2020202020496F6E69616E4D6F9C
:107C2B0064653A2020202020446F7269616E4D6F8D
:107C3B0064653A202020506872796769616E4D6FD8
:107C4B0064653A20202020204C796469616E4D6F69
:107C5B0064653A204D69786F6C796469616E4D6F1C
:107C6B0064653A2020202041656F6C69616E4D6F11
:107C7B0064653A202020204C6F637269616E4E65FB
:107C8B0061706F6C6974616E206D616A6F724E65A5
:107C9B0061706F6C6974616E206D696E6F722020FC
:107CAB0020202020204E696E6520546F6E652020A9
:107CBB0020202020204F637461746F6E6963202035
:107CCB002020202020204F7269656E74616C20206B
:107CDB002020202020204F766572746F6E65202047
:107CEB0020202020202020202050656C6F67202032
:107CFB002020202050656E7461746F6E69636D6116
:107D0B006A6F722050656E7461746F6E69636D6912
:107D1B006E6F722050656E7461746F6E6963202094
:107D2B002020202050726F6D65746865757320205C
:107D3B00202020202020205370616E697368202042
:107D4B0020202053796D6D6574726963616C2020FE
:107D5B00202020202057686F6C65746F6E656C65F2
:107D6B006164696E6757686F6C65746F6E65202010
:107D7B002020202075736572207363616C6503008E
:107D8B0004070000000000000000000300040700CF
:0E7D9B000000000000000000070004070205C1
:107DA900090B0000000000010101010101010101AD
:107DB9000101011E1E1E1E1E1E1E1E1E1E1E1E014E
:107DC900010101010101010101010101010101019A
:107DD900010101010101010CFF00FF01FF02FF0385
:107DE900FF04FF05FF06FF07FF08FF09FF0AFF0B56
:107DF900FF0CFF0DFF0EFF0FFF10FF11FF12FF1306
:107E0900FF14FF15FF16FF17FF18FF19FF1AFF1BB5
:107E1900FF1CFF1DFF1EFF1FC2A5C2A4C295C2A35E
:107E2900E55020160274FF7F083392A6D2A3C2A39D
:107E3900DFF7B2A50000C2A5E55120160274FF794B
:107E4900083392A6C2A3D2A3D9F7D2A40000C2A430
:107E590022C2A6D2A67908C2A3A2A733D2A3D9F770
:107E6900F56AC2A6D2A67908C2A3A28033D2A3D941
:107E7900F7F56B22900166E0B40303027E9150FB93
:107E8900900168E0B4050122900166E0B40701227F
:107E9900B4080122E56B20E50122E56B20E6012209
:107EA900127ECE127F51127FD41280571280DA12BD
:107EB900815D1281E01282631282E6128369128364
:107EC900EC12846F22E56B30E10DC217202314D226
:107ED90023127F1DD23222C223201707D217127E06
:107EE900EDD2322220530620541A027EFD127EFD65
:107EF900127F0D2290020E128670E0B2E7F07F0029
:107F090012888C229004C3128699E0B2E7F07F00B0
:107F19001288972220530620541C027F2D127F2D90
:107F2900127F3F22203A2090020E1286707400F0D0
:107F39007F0012880822203B0E9004C31286997490
:107F490000F07F001288BA22E56B30E20DC21820DA
:107F59002414D224127FA0D23222C224201807D29C
:107F690018127F70D2322220530620541A027F80C1
:107F7900127F80127F902290020F128670E0B2E782
:107F8900F07F0112888C229004C4128699E0B2E72E
:107F9900F07F011288972220530620541C027FB0DB
:107FA900127FB0127FC222203A2090020F128670EF
:107FB9007400F07F0112880822203B0E9004C4123D
:107FC90086997400F07F011288BA22E56B30E30DBF
:107FD900C219202514D225128023D23222C225208B
:107FE9001907D219127FF3D2322220530620541ACC
:107FF90002800312800312801322900210128670ED
:10800900E0B2E7F07F0212888C229004C5128699AB
:10801900E0B2E7F07F021288972220530620541C11
:1080290002803312803312804522203A20900210B8
:108039001286707400F07F0212880822203B0E908D
:1080490004C51286997400F07F021288BA22E56A83
:1080590030E00DC21A202614D2261280A6D232226E
:10806900C226201A07D21A128076D232222053064B
:1080790020541A028086128086128096229002115C
:10808900128670E0B2E7F07F0312888C229004C652
:10809900128699E0B2E7F07F0312889722205306EF
:1080A90020541C0280B61280B61280C822203A20C1
:1080B9009002111286707400F07F03128808222042
:1080C9003B0E9004C61286997400F07F031288BA99
:1080D90022E56A30E10DC21B202714D2271281291B
:1080E900D23222C227201B07D21B1280F9D2322298
:1080F90020530620541A028109128109128119227A
:10810900900212128670E0B2E7F07F0412888C2286
:0E8119009004C7128699E0B2E7F07F04128846
:10812700972220530620541C02813912813912816B
:108137004B22203A209002121286707400F07F04BE
:1081470012880822203B0E9004C71286997400F00B
:108157007F041288BA22E56A30E20DC21C20281477
:10816700D2281281ACD23222C228201C07D21C127C
:10817700817CD2322220530620541A02818C12812C
:108187008C12819C22900213128670E0B2E7F07F76
:108197000512888C229004C8128699E0B2E7F07F16
:1081A700051288972220530620541C0281BC128195
:1081B700BC1281CE22203A209002131286707400DE
:1081C700F07F0512880822203B0E9004C81286997A
:1081D7007400F07F051288BA22E56B30E40DC21DEA
:1081E700202914D22912822FD23222C229201D0718
:1081F700D21D1281FFD2322220530620541A028246
:108207000F12820F12821F22900214128670E0B2A0
:10821700E7F07F0612888C229004C9128699E0B293
:10822700E7F07F061288972220530620541C02820B
:108237003F12823F12825122203A20900214128666
:10824700707400F07F0612880822203B0E9004C944
:108257001286997400F07F061288BA22E56A30E325
:108267000DC21E202A14D22A1282B2D23222C22A68
:10827700201E07D21E128282D23222205306205499
:108287001A0282921282921282A2229002151286FA
:1082970070E0B2E7F07F0712888C229004CA12863A
:1082A70099E0B2E7F07F07128897222053062054FF
:1082B7001C0282C21282C21282D422203A20900269
:1082C700151286707400F07F0712880822203B0E73
:1082D7009004CA1286997400F07F071288BA22E5C3
:1082E7006A30E40DC21F202B14D22B128335D232F1
:1082F70022C22B201F07D21F128305D232222053FE
:108307000620541A02831512831512832522900220
:1083170016128670E0B2E7F07F0812888C2290046C
:10832700CB128699E0B2E7F07F0812889722205394
:108337000620541C02834512834512835722203A94
:10834700209002161286707400F07F0812880822A7
:10835700203B0E9004CB1286997400F07F08128898
:10836700BA22E56A30E50DC220202C14D22C1283E4
:10837700B8D23222C22C202007D220128388D232D0
:108387002220530620541A0283981283981283A836
:1083970022900217128670E0B2E7F07F0912888CEC
:1083A700229004CC128699E0B2E7F07F09128897F1
:1083B7002220530620541C0283C81283C81283DA72
:1083C70022203A209002171286707400F07F09125B
:1083D700880822203B0E9004CC1286997400F07F07
:1083E700091288BA22E56A30E60DC221202D14D27F
:1083F7002D12843BD23222C22D202107D221128492
:108407000BD2322220530620541A02841B12841BDB
:1084170012842B22900218128670E0B2E7F07F0ACE
:1084270012888C229004CD128699E0B2E7F07F0A79
:108437001288972220530620541C02844B12844B27
:1084470012845D22203A209002181286707400F080
:108457007F0A12880822203B0E9004CD1286997459
:1084670000F07F0A1288BA22E56A30E70DC222209F
:108477002E14D22E1284BED23222C22E202207D22E
:108487002212848ED2322220530620541A02849E4E
:0E84970012849E1284AE22900219128670E0AA
:1084A500B2E7F07F0B12888C229004CE128699E0F9
:1084B500B2E7F07F0B1288972220530620541C0246
:1084C50084CE1284CE1284E022203A209002191222
:1084D50086707400F07F0B12880822203B0E9004F2
:1084E500CE1286997400F07F0B1288BA2230321BA7
:1084F500B4080A9006A3124BEFE56C04F0128552FE
:1085050012851B125713125ED1C2322212851B121D
:108515005713125ED12212852212853A2290020E3D
:1085250012865479007B3CE030E70109A3DBF8E9CA
:1085350090029AF0229004C312866279007B3CE097
:1085450030E70109A3DBF8E990054FF02220540933
:1085550090020E1286700285649004C3128699E01B
:1085650020E709E550D2E1F550028577E550C2E1F3
:10857500F550A3E020E709E550D2E2F55002858BDE
:10858500E550C2E2F550A3E020E709E550D2E3F556
:108595005002859FE550C2E3F550A3E020E709E5C9
:1085A50050D2E4F5500285B3E550C2E4F550A3E09E
:1085B50020E709E550D2E6F5500285C7E550C2E649
:1085C500F550A3E020E709E550D2E7F5500285DB39
:1085D500E550C2E7F550A3E020E709E551D2E0F503
:1085E500510285EFE551C2E0F551A3E020E709E529
:1085F50051D2E1F551028603E551C2E1F551A3E0FF
:1086050020E709E551D2E2F551028617E551C2E2AC
:10861500F551A3E020E709E551D2E4F55102862B97
:10862500E551C2E4F551A3E020E709E551D2E6F5AD
:108635005102863FE551C2E6F551A3E020E709E581
:1086450051D2E7F551028653E551C2E7F55122C3F0
:10865500E582956CF582E5839400F58322C3E58276
:10866500956FF582E5839400F5832212865405A261
:10867500900164E075F00CA4240C05A28582378571
:1086850083387837F53B753C00793B120386868243
:108695000886832212866205A2900164E075F00CBB
:1086A500A4240C05A28582378583387837F53B7578
:1086B5003C00793B120386868208868322900166F8
:1086C500E0B403030286D650FB900168E0B40501CF
:1086D50022128715E56B30E603C23822E56A30E4DD
:1086E5000630E616C2382230380122D238900164AD
:1086F500E014120AFCF01285522230380122D238D9
:10870500900164E004120AFCF012871512855222CA
:10871500900164E0B40009E551D2E3D2E5F55122B8
:10872500B40109E551C2E3D2E5F55122B40209E5E8
:1087350051C2E3C2E5F55122E551D2E3C2E5F55157
:1087450022E56B30E603C23922E56B30E403C2391A
:108755002230390122D23920530F205406B23A1261
:10876500877922B23B12879E22B23A128779B23BB1
:1087750012879E22203A1BE550D2E0F5504350DE89
:108785004351D712963ED232856C6D90020174002A
:10879500F022E550C2E0F55022203B1BE550D2E027
:1087A500F5504350DE4351D712964AD232856F6E4B
:1087B5009004B67400F022E550C2E0F55022203A4C
:1087C50007E550D2E0F55022E550C2E0F5502220F1
:1087D5003B07E550D2E0F55022E550C2E0F55022C6
:0287E50020541E
:1087E700041287C3221287D4221288812FFF900296
:1087F70001E0128866EFF0900201E004120D7FF0AD
:1088070022900201E0FC1288812FF57C7B00900109
:10881700E8A3E00BB57CFA8C7C05A2EB1288660511
:10882700A2EBB57C08E57C14900201F02205A2E0DA
:10883700A305A2F0A30B028828900201E0FB900198
:10884700E9E0256CC3956DF0A3DBF6856C6D22908E
:108857000201E0FB9001E9E0256CF0A3DBF922902F
:1088670001E98582378583387837F53B753C007990
:108877003B120386868208868322900164E075F0A6
:108887000CA4240C2220E704128808221287F02265
:1088970020E7041288BA221288A2221288812FFFA9
:1088A7009004B6E0128918EFF09004B6E004120DB8
:1088B7007FF0229004B6E0FC1288812FF57C7B00C4
:1088C70090049DA3E00BB57CFA8C7C05A2EB128982
:1088D7001805A2EBB57C08E57C149004B6F02205D8
:1088E700A2E0A305A2F0A30B0288DA9004B6E0FB8E
:1088F70090049EE0256FC3956EF0A3DBF6856F6E3F
:10890700229004B6E0FB90049EE0256FF0A3DBF90C
:108917002290049E8582378583387837F53B753CEE
:1089270000793B120386868208868322753D00C242
:1089370000C283C2819000427439F0A3741DF0A372
:108947007450F0A3746CF0A37479F0A3740CF0A3C3
:108957007401F0A37406F0E53DB408FB753D00D241
:108967000022E53DB41023200120D201C28174C04A
:10897700F954F053800F4280D282C282E9C454F086
:1089870053800F4280D282C28222E53DB42021C2A9
:10899700817480F954F053800F4280D282C282E9F9
:1089A700C454F053800F4280D282C282753D0022A8
:1089B700C201A2009281900042E582253DF582E046
:1089C700F954F053800F4280D282C282E9C454F036
:1089D70053800F4280D282C282053D2212036A224F
:1089E70012036A12036A12036A12036A12036A12F3
:1089F700036A12036A22C2821289E31289E3C281DF
:108A0700C28312036AD282C287C286D285D28412F7
:108A1700036AC2821289E3C281C28312036AD282C5
:108A2700C287C286D285D28412036AC2821289E3C0
:108A3700C281C28312036AD282C287C286D285D21A
:108A47008412036AC2821289E3C281C28312036A53
:108A5700D282C287C286D285C28412036AC28212B8
:108A670089E3C281C28312036AD282C287C286D2D5
:108A770085C28412036AC2821289E3C281C2831249
:108A8700036AD282D287C286C285C28412036AC2AF
:108A9700821289E3C281C28312036AD282C287C269
:108AA70086C285C28412036AC2821289E3C281C266
:108AB7008312036AD282D287D286D285C2841203F6
:108AC7006AC2821289E3C281C28312036AD282C256
:108AD70087C286C285C28412036AC2821289E3C230
:108AE70081C28312036AD282C287C286C285D284B8
:108AF70012036AC2821289E3C281C28312036AD255
:108B070082C287C286C285C28412036AC282128960
:108B1700E3C281C28312036AD282C287D286D28518
:108B2700C28412036AC2821289E3D2002205A2E438
:108B370093A305A2F0A3DBF505A22290675A05A22D
:108B47009000427B20028B3490677A05A290004206
:0E8B57007B20028B349067CA05A29000427BFF
:108B650020028B342430F02275F00A84AFF075F0C2
:108B75000A84E5F02430F0EF2430A3F02275F00AE2
:108B850084AFF075F00A842430F0E5F02430A3F0CA
:108B9500EF2430A3F022128B82A3742CF0EE243044
:108BA500A3F022D281C28312036AD282D287D286EF
:108BB500D285D28412036AC2821289E3D281C2832A
:108BC50012036AD282D287D286D285D28412036AF0
:108BD500C2821289E322128B5C12036A12036A12A3
:108BE500036A12036A12036A12036A12036A128B7A
:108BF500427550DB7551FF12036A12036A7550CF37
:108C05007551FF12036A12036A7550DF7551FE1222
:108C1500036A12036A7550DF7551FB12036A12036A
:108C25006A7550DF7551BF12036A12036A7550DF0A
:108C350075517F12036A12036A7550DF7551EF1281
:108C4500036A12036A7550DF7551FD12036A120338
:108C55006A75505F7551FF12036A12036A75509F5A
:108C65007551FF12036A12036A7550D77551FF12C9
:108C7500036A12036A7550DD7551FF12036A120308
:108C85006A7550DF7551FF128B4F4352FF12036A0D
:108C950012036A12036A12036A12036A12036A1242
:108CA500036A12036A12036A12036A12036A120341
:108CB5006A12036A12036A12036A12036A12036ACA
:108CC50012036A12036A12036A12036A12036A1212
:108CD500036A12036A12036A12036A12036A120311
:108CE5006A12036A12036A535200128B5C12036AFA
:108CF50012036A12036A12036A22E56B30E001224D
:108D0500435020E550C2E2F550E551C2E0F55190DF
:108D1500679A05A29000427B10128B349067AA05D2
:108D2500A29000527B10128B34E56B30E0FBE56BB3
:108D350030E20630E417028D339067BA05A2900041
:108D4500527B10128B3412036A128ED522E56B30DA
:108D5500E4FB12036A12036A22E5D220E0FBE0A3DA
:108D650005A2C2AF75D202F075D200D2AFA305A29B
:108D7500DBE722E5D220E0FBC2AF75D202E075D277
:108D850000D2AFA305A2F0A305A2DBE722900180E4
:108D9500128F7305A27B0D90065305A2128D7822C2
:108DA500900197128F7305A27B0D90066005A212A4
:108DB5008D7822900181128FE405A27B0D90066DBE
:108DC50005A2128D7822900198128FE405A27B0DE1
:108DD50090067A05A2128D782290000005A27B0DDF
:108DE50090065305A2128D7890000005A27B0D9088
:108DF500066005A2128D789000D005A27B0D900625
:108E05006D05A2128D789000D005A27B0D90067A93
:108E150005A2128D782290029E05A27B3190068BC9
:108E250005A2128D78229002CF05A27B7690017360
:108E350005A2128D7822900178128FA005A27B02DF
:108E450090018205A2128D782290018F128FA005C4
:108E5500A27B0290019905A2128D78229001A2129F
:108E65004697128FA005A29001D31248FF7B0205F9
:108E7500A2128D78227B0D90065305A29000000565
:108E8500A2128D5E227B0D90066D05A29000D00585
:108E9500A2128D5E227B3190068B05A290029E0563
:108EA500A2128D5E227B7690017305A29002CF05FA
:108EB500A2128D5E22E5D220E0FBEA930A05A2C24A
:108EC500AF75D202F075D200D2AFA305A2DBE622C0
:0E8ED500128EE8128EFC128F10128F2412974C
:108EE30014128EAA2290000005A27C10907D897B2B
:108EF3000D7A00128EBADCF4229000D005A27C1009
:108F0300907DA37B0D7A00128EBADCF42290029E30
:108F130005A27C01907DB07B317A00128EBADCF41D
:108F2300229001A07B7F7980128F3FA3DBFA90010F
:108F3300A17B7F7900128F3FA3DBFA22E5D220E0E9
:108F4300FBE9C2AF75D202F075D200D2AFA322E023
:108F53001475F00DA4900000858237858338783727
:108F6300F53B753C00793B12038686820886832293
:108F7300E0B42B03028F7E50FB742BC3942B75F04C
:108F83000DA49000008582378583387837F53B75CB
:108F93003C00793B120386868208868322E0C394D1
:108FA3008075F002A49001A08582378583387837D5
:108FB300F53B753C00793B12038686820886832243
:108FC300E01475F00DA49000D0858237858338783E
:108FD30037F53B753C00793B12038686820886830E
:108FE30022E0B43703028FEF50FB7437C394377515
:108FF300F00DA49000D08582378583387837F53B10
:10900300753C00793B120386868208868322E0142E
:1090130075F004A490901B739001A0229001E022AC
:1090230090021E2290022E2290023E2290024E2295
:1090330090025E2290026E2290027E2290028E2285
:109043008582378583387837900163E01475F002A1
:10905300A4F53B753C00793B120386868208868320
:1090630022C2A5C2A4C295C2A3E5527F083392A629
:10907300D2A3C2A3DFF7B2950000C2952220360126
:1090830022C2364350DE4351D7E550C2E0F550309B
:10909300530BD23AD23B1290AF1291642220540662
:1090A300D23A1290AF22D23B1291642212963E9092
:1090B30002017400F0856C6D900180E0B42B030213
:1090C30090E750FB1475F005A4FB90739993FA0B8A
:1090D300EB9305A212914305A2DAF412910B1288C5
:1090E30056D23222128D92900653E0FA70061296EF
:1090F3003ED23222A3E005A212914305A2DAF51271
:109103009133128856D23222900180E01475F00513
:10911300A4FB9001E905A290739993FAFF0BEB93DB
:10912300240C05A2F0A305A2DAF3EF900201F022CA
:109133009001E905A29006531291F0900201F022EA
:1091430090021A8582378583387837F53B753C0062
:10915300793B120386868208868374FFF012997521
:109163002212964A9004B67400F0856F6E900197B0
:10917300E0B42B0302919C50FB1475F005A4FB9003
:10918300739993FA0BEB9305A212920105A2DAF4F9
:109193001291B8128908D23222128DA5900660E08E
:1091A300FAA3E005A212920105A2DAF51291E012E8
:1091B3008908D23222900197E01475F005A4FB9040
:1091C300049E05A290739993FAFF0BEB93240C056D
:1091D300A2F0A305A2DAF3EF9004B6F02290049E66
:1091E30005A29006601291F09004B6F022E0FAFF17
:1091F300A3E0240C05A2F0A305A2DAF4EF22900465
:10920300CF8582378583387837F53B753C00793BCA
:10921300120386868208868374FFF0129975229062
:10922300029AE0700122B4040302923340FB7404F7
:109233001475F003A490923C73029248029269025F
:1092430092980292BD9006BCE0FD9001E9E02D905A
:0E92530006BDF0240C9006BEF0240C9006BF61
:10926100F0240C9006C0F0227A029006BCE0FD903A
:1092710006BD05A29001E9E02DA305A2F0A305A278
:10928100DAF59006BDE0240C9006BFF09006BEE032
:10929100240C9006C0F0227A039006BCE0FD9006F3
:1092A100BD05A29001E9E02DA305A2F0A305A2DA74
:1092B100F59006BDE0240C9006C0F0227A049006D9
:1092C100BCE0FD9006BD05A29001E9E02DA305A239
:1092D100F0A305A2DAF5229006BDE012061B8582F5
:1092E100488583499006BEE012061B85824A858324
:1092F1004B90017FE0B4020D9006BFE012061B8582
:10930100824C85834D900196E0B4020D9006C0E039
:1093110012061B85824E85834F2290029AE0B4008B
:109321000412936322B4010D1293701293E7129405
:109331003412948122B4020D1293701293BD1294CF
:109341003412948122B4030D1293701293BD1294BE
:109351000A129481221293701293BD12940A1294EC
:10936100572212939A1293E7129434129481221283
:10937100939A9006BDE0FF7492120E079006BCE02E
:109381002F2424C2E79006C1F0120E077464120E56
:10939100079006C5E0D2E0F0229006C5E020E0018A
:1093A100229006C1E0FF7492120E07EF120E0774AD
:1093B10000120E079006C5E0C2E0F0221293E7907A
:1093C10006BEE0FF7492120E079006BCE02F242423
:1093D100C2E79006C2F0120E077464120E079006DF
:1093E100C5E0D2E1F0229006C5E020E1012290061D
:1093F100C2E0FF7492120E07EF120E077400120EF4
:10940100079006C5E0C2E1F0221294349006BFE055
:10941100FF7492120E079006BCE02F2424C2E7903D
:1094210006C3F0120E077464120E079006C5E0D24F
:10943100E2F0229006C5E020E201229006C3E0FF9F
:109441007492120E07EF120E077400120E079006A7
:10945100C5E0C2E2F0221294819006C0E0FF74924E
:10946100120E079006BCE02F2424C2E79006C4F038
:10947100120E077464120E079006C5E0D2E3F022C3
:109481009006C5E020E301229006C4E0FF74921229
:109491000E07EF120E077400120E079006C5E0C208
:1094A100E3F02220370122C2374350DE4351D7E592
:1094B10050C2E0F55030530BD23AD23B1294D31242
:1094C10094EB22205406D23A1294D322D23B129426
:1094D100EB2212963E9002017400F0856C6D12959C
:1094E10003129514128856D2322212964A9004B66B
:1094F1007400F0856F6E12958912959A128908D2BF
:109501003222900181E0B4370412953B2250FA12C5
:10951100952B22900181E0B4370712953B12956A91
:109521002250F712960F1295502212960F0BEB93C1
:1095310005A212914305A2DAF422128DB890066DAC
:10954100E0FAFFA3E005A212914305A2DAF5220594
:10955100A29001E905A20BEB93240C05A2F0A3054F
:10956100A2DAF3EF900201F02290066DE0FFFA0516
:10957100A29001E905A2A3E0240C05A2F0A305A293
:10958100DAF4EF900201F022900198E0B43704126E
:1095910095C12250FA1295B122900198E0B4370793
:1095A1001295C11295F02250F712960F1295D622FC
:1095B10012960F0BEB9305A212920105A2DAF42287
:1095C100128DCB90067AE0FAFFA3E005A212920178
:0E95D10005A2DAF52205A290049E05A20BEB7E
:1095DF0093240C05A2F0A305A2DAF3EF9004B6F0E2
:1095EF002290067AE0FFFA05A290049E05A2A3E05E
:1095FF00240C05A2F0A305A2DAF4EF9004B6F02232
:10960F00B41303029617500690775C029634B42673
:10961F00030296255009907853C394130296349001
:10962F007949C394261475F00DA4FB93FAFF2274A5
:10963F00007998900202F0A3D9FC227400799890D7
:10964F0004B7F0A3D9FC227908F0A3D9FC22740146
:10965F009001A212965674039001AA1296567406A0
:10966F009001B212965674069001BA12965674046F
:10967F009001C312965674039001CB129656227422
:10968F000090014B12965622740090013B12965691
:10969F0022740090014312965622791190007A7429
:1096AF0000F0A37400F0A3D9F6799990009C740090
:1096BF00F0A3D9FC22790A9006D07401F0A3D9FC4B
:1096CF00229006530296D990066074057900F07BBC
:1096DF000CA3E9F009DBFA2290066D0296F09006D2
:1096EF007A74057900F07B0CA3E9F009DBFA900698
:1096FF008B12970B2290069712970B227B0C7401FB
:10970F00F0A3DBFC22746E900173F074019001746E
:10971F00F0900175F0900184F0741190017BF0745A
:10972F000190018AF090017EF0740290017FF07435
:10973F000190017CF090017DF07403900179F07439
:10974F0006900185F0900186F0740490017AF07410
:10975F0003900187F07401900176F0740290017804
:10976F00F07400900177F07400900188F004F074A9
:10977F0001900180F07401900181F0740190018BD0
:10978F00F090018CF090019BF07411900192F074A5
:10979F00019001A1F0900195F07402900196F07480
:1097AF0001900193F0900194F07403900190F07484
:1097BF000690019CF090019DF07404900191F0745B
:1097CF000390019EF0740190018DF0740290018F4F
:1097DF00F0740090018EF0740090019FF004F0740B
:1097EF0001900197F0900198F074029001E3F090CE
:1097FF0001E4F01296D01296D61296E71296ED90DB
:10980F0001E57400F09001E67402F0C25AD2507470
:10981F00029001E7F074029001E8F02290017BE0E2
:10982F0014B41009C3940F7980C9C3992250F575E8
:10983F00F003A4909846730298C10298C10299064A
:10984F0002990B02991002991502991A02991F0297
:10985F0099240299290298C10298C90298D10298B5
:10986F00DB0298E31298EF900192E014B41009C351
:10987F00940F7980C9C3992250F575F003A490987D
:10988F0091730298C10298C102992E0299330299DD
:10989F003802993D02994202994702994C02995117
:1098AF000298C10298C90298D10298DB0298E3127C
:1098BF0098EF126602547FD2E022126602543F24C0
:1098CF00402212660275F00584244C22126602545F
:1098DF001F246022126602541F75F0028424702226
:1098EF0012660254016008126602541F2454221299
:1098FF006602540F2470227402029956740302995F
:10990F0056740402995674050299567406029956B4
:10991F00740702995674080299567409029956747D
:10992F000202995D740302995D740402995D7405D6
:10993F0002995D740602995D740702995D740802BD
:0E994F00995D740902995D900188F00299619A
:10995D0090019FF0F57CA3E004B57C067400F074D3
:10996D007F2250F8F074642222F9900041E0B40097
:10997D00012290003FE0900000F582E9F090003F59
:10998D00E004B43F027400F0900041E014F022C2F4
:10999D00AC900041E0B43E03D2AC2204F090004004
:1099AD00E0900000F582E0F9900040E004B43F0241
:1099BD007400F0D2ACE9120E4102999C304FD0C226
:1099CD004F22900689E020E00122C2E0F01299E4D6
:1099DD00129A13129A3A229001E5E030E00122C268
:1099ED00AD1204D0D2AD12047475F00A8404120BBA
:1099FD00C1F57C9006C7E0B57C0122E57CF09001B5
:109A0D0074F012851122C2AD1204C4D2AD120474C9
:109A1D0075F03F8404120CC1F57C9006C8E0B57C4E
:109A2D000122E57CF0900176F0128511229006CD91
:109A3D00E01475F003A4909A4773029ABB029AF052
:109A4D00029B10029B2B029B4D029B5A029B6702AD
:109A5D009B74029B91029BB8029BC4029BE2029CE9
:109A6D0007029C14029C21029C2E029C4B029C69B5
:109A7D00029C8E029C9B029CA8029CB5029CD20269
:109A8D009CF0029D15029D22029D2F029D3C029D80
:109A9D0059029D77029D9C029DA9029DB6029DC310
:109AAD00029AD7C2AD1204B8D2AD12047422129A22
:109ABD00B075F00284120C0DF57C9006CBE0B57CF0
:109ACD000122E57CF0900177F022129AB0120A542F
:109ADD0014F57C9006CBE0B57C0122E57CF090017D
:109AED0073F022129AB075F01C8404120BE7F57C0A
:109AFD009006CBE0B57C0122E57CF0900175F0126B
:109B0D00851122129AB0F57C9006CBE0B57C01222E
:109B1D00E57CF0900178F0122E4B122D6922129AED
:109B2D00B075F00F8404120CAEF57C9006CBE0B549
:109B3D007C0122E57CF0900179F0122F10D24A229F
:109B4D00129AB075F03384042401029B36129AB038
:109B5D0075F03384042407029B36129AB075F040D9
:109B6D008404240D029B36129AB075F018840412E9
:109B7D000CD4F57C9006CBE0B57C0122E57CF09011
:109B8D00017AF022129AB075F0028404120AE97972
:109B9D007FC9C3992411120C1DF57C9006CBE0B53D
:109BAD007C0122E57CF090017BF022129AB075F0D9
:109BBD0012842403029BA6129AB0F57C9006CBE08A
:109BCD00B57C0122E57CF09001A2F0900167740153
:109BDD00F012481922129AB075F00F8404120CAECF
:109BED00F57C9006CBE0B57C0122E57CF09001AAD6
:109BFD00F079019001C2E049F022129AB075F0336C
:109C0D0084042401029BED129AB075F03384042470
:109C1D0007029BED129AB075F0408404240D029B4F
:109C2D00ED129AB075F0188404120CD4F57C9006E0
:109C3D00CBE0B57C0122E57CF09001C3F022129AB5
:109C4D00B0F57C9006CBE0B57C0122E57CF090016F
:109C5D00A3F09001677402F012481922129AB075A0
:109C6D00F00F8404120CAEF57C9006CBE0B57C01B0
:109C7D0022E57CF09001ABF079029001C2E049F051
:109C8D0022129AB075F03384042401029C74129A46
:109C9D00B075F03384042407029C74129AB075F0E9
:109CAD00408404240D029C74129AB075F01884F54A
:109CBD007C9006CBE0B57C0122E57C04120CD4F03F
:0E9CCD009001C4F022129AB0F57C9006CBE014
:109CDB00B57C0122E57CF09001A4F0900167740340
:109CEB00F012481922129AB075F00F8404120CAEC0
:109CFB00F57C9006CBE0B57C0122E57CF09001ACC5
:109D0B00F079049001C2E049F022129AB075F03359
:109D1B0084042401029CFB129AB075F03384042452
:109D2B0007029CFB129AB075F0408404240D029C30
:109D3B00FB129AB075F0188404120CD4F57C9006C3
:109D4B00CBE0B57C0122E57CF09001C5F022129AA4
:109D5B00B0F57C9006CBE0B57C0122E57CF0900160
:109D6B00A5F09001677404F012481922129AB0758D
:109D7B00F00F8404120CAEF57C9006CBE0B57C01A1
:109D8B0022E57CF09001ADF079089001C2E049F03A
:109D9B0022129AB075F03384042401029D82129A28
:109DAB00B075F03384042407029D82129AB075F0CB
:109DBB00408404240D029D82129AB075F01884041D
:109DCB00120CD4F57C9006CBE0B57C0122E57CF03F
:109DDB009001C6F022900689E020E30122C2E3F055
:109DEB00129DF5129E27129E4E22C2AD1204E8D28E
:109DFB00AD12047475F00A8404120BC1F57C900645
:109E0B00C9E0B57C0122E57CF090018BF09001E577
:109E1B00E030E00412A2712212851122C2AD1204AD
:109E2B00ACD2AD12047475F03F84F57C9006CAE099
:109E3B00B57C0122E57C04120CC1F090018DF0126F
:109E4B008511229006CEE01475F003A4909E5B73EF
:109E5B00029ECC029EE8029F08029F23029F4502AE
:109E6B009F52029F5F029F6C029F89029FB0029FCD
:109E7B00BC029FDA029FFF02A00C02A01902A026CF
:109E8B0002A04302A06102A08602A09302A0A0023E
:109E9B00A0AD02A0CA02A0E802A10D02A11A02A164
:109EAB002702A13402A15102A16F02A19402A1A128
:109EBB0002A1AE02A1BBC2AD1204DCD2AD1204747E
:109ECB0022129EC175F00284120C0DF57C9006CC0B
:109EDB00E0B57C0122E57CF090018EF022129EC150
:109EEB0075F01C8404120BE7F57C9006CCE0B57C76
:109EFB000122E57CF090018CF012851122129EC19B
:109F0B00F57C9006CCE0B57C0122E57CF090018FCE
:109F1B00F01238201237AD22129EC175F00F840457
:109F2B00120CAEF57C9006CCE0B57C0122E57CF002
:109F3B00900190F0123878D24B22129EC175F033FB
:109F4B0084042401029F2E129EC175F033840424D5
:109F5B0007029F2E129EC175F0408404240D029FB0
:109F6B002E129EC175F0188404120CD4F57C900649
:109F7B00CCE0B57C0122E57CF0900191F022129EA1
:109F8B00C175F0028404120AE9797FC9C3992411BF
:109F9B00120C1DF57C9006CCE0B57C0122E57CF023
:109FAB00900192F022129EC175F012842403029F3D
:109FBB009E129EC1F57C9006CCE0B57C0122E57C1F
:109FCB00F09001A6F09001677405F0124819221267
:109FDB009EC175F00F8404120CAEF57C9006CCE09C
:109FEB00B57C0122E57CF09001AEF079109001C2B6
:109FFB00E049F022129EC175F03384042401029FC4
:10A00B00E5129EC175F03384042407029FE5129E6E
:10A01B00C175F0408404240D029FE5129EC175F0BA
:10A02B00188404120CD4F57C9006CCE0B57C01228C
:10A03B00E57CF09001C7F022129EC1F57C9006CC16
:0EA04B00E0B57C0122E57CF09001A7F09001C9
:10A05900677406F012481922129EC175F00F840424
:10A06900120CAEF57C9006CCE0B57C0122E57CF0C3
:10A079009001AFF079209001C2E049F022129EC10F
:10A0890075F0338404240102A06C129EC175F0336B
:10A099008404240702A06C129EC175F04084042434
:10A0A9000D02A06C129EC175F0188404120CD4F52F
:10A0B9007C9006CCE0B57C0122E57CF09001C8F0EB
:10A0C90022129EC1F57C9006CCE0B57C0122E57C8C
:10A0D900F09001A8F09001677407F0124819221254
:10A0E9009EC175F00F8404120CAEF57C9006CCE08D
:10A0F900B57C0122E57CF09001B0F079409001C275
:10A10900E049F022129EC175F0338404240102A0B3
:10A11900F3129EC175F0338404240702A0F3129E42
:10A12900C175F0408404240D02A0F3129EC175F09C
:10A13900188404120CD4F57C9006CCE0B57C01227D
:10A14900E57CF09001C9F022129EC1F57C9006CC05
:10A15900E0B57C0122E57CF09001A9F090016774DB
:10A1690008F012481922129EC175F00F8404120CCE
:10A17900AEF57C9006CCE0B57C0122E57CF090013F
:10A18900B1F079809001C2E049F022129EC175F0C8
:10A19900338404240102A17A129EC175F033840428
:10A1A900240702A17A129EC175F0408404240D028D
:10A1B900A17A129EC175F0188404120CD4F57C9012
:10A1C90006CCE0B57C0122E57CF09001CAF0229032
:10A1D9000689E020E40122C2E4F0D25F12A1F21262
:10A1E900A20E12922212931B22C2AD120500D2AD09
:10A1F90012047475F01584F57C9006BCE0B57C01F9
:10A2090022E57CF022C2AD1204F4D2AD12047475B9
:10A21900F0178404F57C9006C6E0B57C0122E57C44
:10A22900F0F57C9006BBE0B57C0990016FE57CF008
:10A23900D2582250F522900689E020E20122C2E29A
:10A24900F09001E5E0B2E0F020E00412A28D2212C4
:10A25900A269229001E5E020E003D29122C2912275
:10A26900900174E090068AF0C29190018BE0B419D4
:10A279000302A28520E0041402A28504900174F06F
:10A2890012851122D29190068AE0900174F012850C
:10A29900112243B71843B812758790758922758DB5
:10A2A900F8758BF8D28E759850C299C298D2ACC203
:10A2B9001175532875540475557D75560290FF9C88
:10A2C9008582CA8583CB8582CC8583CD43C804D258
:10A2D900ADD2AF2243B74043B8408541EA8542FA3F
:10A2E90043D90143DA4975570875580CD2DED2AE05
:10A2F90022439C00439D1D43B10122C0E0C0D0E52B
:10A3090082C0E0E583C0E0900689E59EF0539EE2B5
:10A31900D0E0F583D0E0F582D0D0D0E032C0E0C003
:10A32900D030DF07C2DFD0D0D0E032C2D8E5EA258D
:10A3390041F5EAE5FA3542F5FAD5570B755708D2D2
:10A3490009D5580375580CD0D0D0E032C0E0C0D040
:10A35900E582C0E0E583C0E0C2D4D2D3309911C20E
:10A3690011C299D0E0F583D0E0F582D0D0D0E032A7
:10A37900309807C298E599129976D0E0F583D0E034
:10A38900F582D0D0D0E032C0E0C0D0E582C0E0E5AF
:10A3990083C0E0D2D4C2D3C2CF201212D55D0F75CB
:10A3A9005DFFD55E09855B5D855C5E122003201328
:10A3B90012D5630F7563FFD564098561638562648E
:0EA3C9001222DBD5533B75532812050C128966
:10A3D7006912064B12065C129064D5542675540612
:10A3E700127E5AB216127E21D55518755532C205FE
:10A3F700900160E0600214F0D55608755603D20547
:10A4070012664CD0E0F583D0E0F582D0D0D0E032B0
:00000001FF
